 wavedev2_sgtl5000

 Timestamp is 4fb05c76 (Mon May 14 13:14:30 2012)

 Preferred load address is 10000000

 Start         Length     Name                   Class
 0001:00000000 00000004H .CRT$XCA                CODE
 0001:00000004 00000004H .CRT$XCZ                CODE
 0001:00000008 00000004H .CRT$XIA                CODE
 0001:0000000c 00000004H .CRT$XIZ                CODE
 0001:00000010 00000004H .CRT$XPA                CODE
 0001:00000014 00000004H .CRT$XPZ                CODE
 0001:00000018 00000004H .CRT$XTA                CODE
 0001:0000001c 00000004H .CRT$XTZ                CODE
 0001:00000020 0000406aH .rdata                  CODE
 0001:0000408c 0000002eH .rdata$debug            CODE
 0001:000040bc 0001587cH .text                   CODE
 0001:00019938 00000078H .xdata                  CODE
 0001:000199b0 00000064H .idata$2                CODE
 0001:00019a14 00000014H .idata$3                CODE
 0001:00019a28 00000160H .idata$4                CODE
 0001:00019b88 00000196H .idata$6                CODE
 0001:00019d20 000000a1H .edata                  CODE
 0002:00000000 00000160H .idata$5                DATA
 0002:00000160 000005f8H .data                   DATA
 0002:00000758 00000068H .bss                    DATA
 0003:00000000 00000c88H .pdata                  DATA

  Address         Publics by Value              Rva+Base       Lib:Object

 0000:00000000       ___safe_se_handler_count   00000000     <absolute>
 0000:00000000       ___safe_se_handler_table   00000000     <absolute>
 0001:00000000       __xc_a                     10001000     corelib0:crt0init.obj
 0001:00000004       __xc_z                     10001004     corelib0:crt0init.obj
 0001:00000008       __xi_a                     10001008     corelib0:crt0init.obj
 0001:0000000c       __xi_z                     1000100c     corelib0:crt0init.obj
 0001:00000010       __xp_a                     10001010     corelib0:crt0init.obj
 0001:00000014       __xp_z                     10001014     corelib0:crt0init.obj
 0001:00000018       __xt_a                     10001018     corelib0:crt0init.obj
 0001:0000001c       __xt_z                     1000101c     corelib0:crt0init.obj
 0001:00000040       ??_C@_1GK@KIEOPOHO@?$AAB?$AAS?$AAP?$AAA?$AAu?$AAd?$AAi?$AAo?$AAI?$AAn?$AAi?$AAt?$AAC?$AAo?$AAd?$AAe?$AAc?$AA?3?$AA?5?$AAI?$AAn?$AAi?$AAt?$AA?5?$AAS?$AAG?$AAT?$AAL?$AA5?$AA0?$AA0?$AA0@ 10001040     bsphwctxt.obj
 0001:000000ac       ??_C@_1M@LCEEOPDH@?$AAI?$AA2?$AAC?$AA1?$AA?3?$AA?$AA@ 100010ac     sgtl5000codec.obj
 0001:000000b8       ??_C@_1FG@POLJNAAL@?$AAS?$AAG?$AAT?$AAL?$AA5?$AA0?$AA0?$AA0?$AAW?$AAr?$AAi?$AAt?$AAe?$AAR?$AAe?$AAg?$AAi?$AAs?$AAt?$AAe?$AAr?$AA?$CI?$AA0?$AAx?$AA?$CF?$AAx?$AA?$CJ?$AA?$DN?$AA0?$AAx?$AA?$CF?$AAx@ 100010b8     sgtl5000codec.obj
 0001:00000110       ??_C@_1FE@MEILOKNP@?$AAS?$AAG?$AAT?$AAL?$AA5?$AA0?$AA0?$AA0?$AAR?$AAe?$AAa?$AAd?$AAR?$AAe?$AAg?$AAi?$AAs?$AAt?$AAe?$AAr?$AA?$CI?$AA0?$AAx?$AA?$CF?$AAx?$AA?$CJ?$AA?$DN?$AA0?$AAx?$AA?$CF?$AAx?$AA?5@ 10001110     sgtl5000codec.obj
 0001:00000168       ??_C@_1EE@MGPNIIMF@?$AAE?$AAr?$AAr?$AAo?$AAr?$AA?0?$AAn?$AAo?$AAt?$AA?5?$AAs?$AAu?$AAp?$AAp?$AAo?$AAr?$AAt?$AAe?$AAd?$AA?5?$AAs?$AAa?$AAm?$AAp?$AAl?$AAe?$AA?5?$AAr?$AAa?$AAt?$AAe?$AA?$AN@ 10001168     sgtl5000codec.obj
 0001:000001ac       ??_C@_1DK@HLMHNKLP@?$AAD?$AAA?$AAP?$AA_?$AAC?$AAO?$AAE?$AAF?$AA_?$AAW?$AAR?$AA_?$AAA?$AA2?$AA_?$AAL?$AAS?$AAB?$AA?5?$AA?$DN?$AA?5?$AA0?$AAx?$AA?$CF?$AAx?$AA?5?$AA?$AN?$AA?6?$AA?$AA@ 100011ac     sgtl5000codec.obj
 0001:000001e8       ??_C@_1DK@HKHCCHKC@?$AAD?$AAA?$AAP?$AA_?$AAC?$AAO?$AAE?$AAF?$AA_?$AAW?$AAR?$AA_?$AAA?$AA2?$AA_?$AAM?$AAS?$AAB?$AA?5?$AA?$DN?$AA?5?$AA0?$AAx?$AA?$CF?$AAx?$AA?5?$AA?$AN?$AA?6?$AA?$AA@ 100011e8     sgtl5000codec.obj
 0001:00000224       ??_C@_1DK@LCNINCAA@?$AAD?$AAA?$AAP?$AA_?$AAC?$AAO?$AAE?$AAF?$AA_?$AAW?$AAR?$AA_?$AAA?$AA1?$AA_?$AAL?$AAS?$AAB?$AA?5?$AA?$DN?$AA?5?$AA0?$AAx?$AA?$CF?$AAx?$AA?5?$AA?$AN?$AA?6?$AA?$AA@ 10001224     sgtl5000codec.obj
 0001:00000260       ??_C@_1DK@LDGNCPBN@?$AAD?$AAA?$AAP?$AA_?$AAC?$AAO?$AAE?$AAF?$AA_?$AAW?$AAR?$AA_?$AAA?$AA1?$AA_?$AAM?$AAS?$AAB?$AA?5?$AA?$DN?$AA?5?$AA0?$AAx?$AA?$CF?$AAx?$AA?5?$AA?$AN?$AA?6?$AA?$AA@ 10001260     sgtl5000codec.obj
 0001:0000029c       ??_C@_1DK@BGEBCJOF@?$AAD?$AAA?$AAP?$AA_?$AAC?$AAO?$AAE?$AAF?$AA_?$AAW?$AAR?$AA_?$AAB?$AA2?$AA_?$AAL?$AAS?$AAB?$AA?5?$AA?$DN?$AA?5?$AA0?$AAx?$AA?$CF?$AAx?$AA?5?$AA?$AN?$AA?6?$AA?$AA@ 1000129c     sgtl5000codec.obj
 0001:000002d8       ??_C@_1DK@BHPENEPI@?$AAD?$AAA?$AAP?$AA_?$AAC?$AAO?$AAE?$AAF?$AA_?$AAW?$AAR?$AA_?$AAB?$AA2?$AA_?$AAM?$AAS?$AAB?$AA?5?$AA?$DN?$AA?5?$AA0?$AAx?$AA?$CF?$AAx?$AA?5?$AA?$AN?$AA?6?$AA?$AA@ 100012d8     sgtl5000codec.obj
 0001:00000314       ??_C@_1DK@NPFOCBFK@?$AAD?$AAA?$AAP?$AA_?$AAC?$AAO?$AAE?$AAF?$AA_?$AAW?$AAR?$AA_?$AAB?$AA1?$AA_?$AAL?$AAS?$AAB?$AA?5?$AA?$DN?$AA?5?$AA0?$AAx?$AA?$CF?$AAx?$AA?5?$AA?$AN?$AA?6?$AA?$AA@ 10001314     sgtl5000codec.obj
 0001:00000350       ??_C@_1DK@NOOLNMEH@?$AAD?$AAA?$AAP?$AA_?$AAC?$AAO?$AAE?$AAF?$AA_?$AAW?$AAR?$AA_?$AAB?$AA1?$AA_?$AAM?$AAS?$AAB?$AA?5?$AA?$DN?$AA?5?$AA0?$AAx?$AA?$CF?$AAx?$AA?5?$AA?$AN?$AA?6?$AA?$AA@ 10001350     sgtl5000codec.obj
 0001:0000038c       ??_C@_1DA@NAOAIKEL@?$AAD?$AAA?$AAP?$AA_?$AAA?$AAV?$AAC?$AA_?$AAD?$AAE?$AAC?$AAA?$AAY?$AA?5?$AA?$DN?$AA?5?$AA0?$AAx?$AA?$CF?$AAx?$AA?5?$AA?$AN?$AA?6?$AA?$AA@ 1000138c     sgtl5000codec.obj
 0001:000003bc       ??_C@_1DC@MPEHOJBC@?$AAD?$AAA?$AAP?$AA_?$AAA?$AAV?$AAC?$AA_?$AAA?$AAT?$AAT?$AAA?$AAC?$AAK?$AA?5?$AA?$DN?$AA?5?$AA0?$AAx?$AA?$CF?$AAx?$AA?5?$AA?$AN?$AA?6?$AA?$AA@ 100013bc     sgtl5000codec.obj
 0001:000003f0       ??_C@_1DI@BOCEKIIM@?$AAD?$AAA?$AAP?$AA_?$AAA?$AAV?$AAC?$AA_?$AAT?$AAH?$AAR?$AAE?$AAS?$AAH?$AAO?$AAL?$AAD?$AA?5?$AA?$DN?$AA?5?$AA0?$AAx?$AA?$CF?$AAx?$AA?5?$AA?$AN?$AA?6?$AA?$AA@ 100013f0     sgtl5000codec.obj
 0001:00000428       ??_C@_1CO@MPJALJFM@?$AAD?$AAA?$AAP?$AA_?$AAA?$AAV?$AAC?$AA_?$AAC?$AAT?$AAR?$AAL?$AA?5?$AA?$DN?$AA?5?$AA0?$AAx?$AA?$CF?$AAx?$AA?5?$AA?$AN?$AA?6?$AA?$AA@ 10001428     sgtl5000codec.obj
 0001:00000458       ??_C@_1CO@MIFKJMFB@?$AAD?$AAA?$AAP?$AA_?$AAM?$AAI?$AAX?$AA_?$AAC?$AAH?$AAA?$AAN?$AA?5?$AA?$DN?$AA?5?$AA0?$AAx?$AA?$CF?$AAx?$AA?5?$AA?$AN?$AA?6?$AA?$AA@ 10001458     sgtl5000codec.obj
 0001:00000488       ??_C@_1DA@KGOOKPEN@?$AAD?$AAA?$AAP?$AA_?$AAM?$AAA?$AAI?$AAN?$AA_?$AAC?$AAH?$AAA?$AAN?$AA?5?$AA?$DN?$AA?5?$AA0?$AAx?$AA?$CF?$AAx?$AA?5?$AA?$AN?$AA?6?$AA?$AA@ 10001488     sgtl5000codec.obj
 0001:000004b8       ??_C@_1EI@BEICHBIO@?$AAD?$AAA?$AAP?$AA_?$AAA?$AAU?$AAD?$AAI?$AAO?$AA_?$AAE?$AAQ?$AA_?$AAT?$AAR?$AAE?$AAB?$AAL?$AAE?$AA_?$AAB?$AAA?$AAN?$AAD?$AA4?$AA?5?$AA?$DN?$AA?5?$AA0?$AAx?$AA?$CF?$AAx@ 100014b8     sgtl5000codec.obj
 0001:00000500       ??_C@_1DK@BNGLBEFC@?$AAD?$AAA?$AAP?$AA_?$AAA?$AAU?$AAD?$AAI?$AAO?$AA_?$AAE?$AAQ?$AA_?$AAB?$AAA?$AAN?$AAD?$AA3?$AA?5?$AA?$DN?$AA?5?$AA0?$AAx?$AA?$CF?$AAx?$AA?5?$AA?$AN?$AA?6?$AA?$AA@ 10001500     sgtl5000codec.obj
 0001:0000053c       ??_C@_1DK@JMEOHBHF@?$AAD?$AAA?$AAP?$AA_?$AAA?$AAU?$AAD?$AAI?$AAO?$AA_?$AAE?$AAQ?$AA_?$AAB?$AAA?$AAN?$AAD?$AA2?$AA?5?$AA?$DN?$AA?5?$AA0?$AAx?$AA?$CF?$AAx?$AA?5?$AA?$AN?$AA?6?$AA?$AA@ 1000153c     sgtl5000codec.obj
 0001:00000578       ??_C@_1DK@MEFANIFN@?$AAD?$AAA?$AAP?$AA_?$AAA?$AAU?$AAD?$AAI?$AAO?$AA_?$AAE?$AAQ?$AA_?$AAB?$AAA?$AAN?$AAD?$AA1?$AA?5?$AA?$DN?$AA?5?$AA0?$AAx?$AA?$CF?$AAx?$AA?5?$AA?$AN?$AA?6?$AA?$AA@ 10001578     sgtl5000codec.obj
 0001:000005b8       ??_C@_1EE@KMKJEIOI@?$AAD?$AAA?$AAP?$AA_?$AAA?$AAU?$AAD?$AAI?$AAO?$AA_?$AAE?$AAQ?$AA_?$AAB?$AAA?$AAS?$AAS?$AA_?$AAB?$AAA?$AAN?$AAD?$AA0?$AA?5?$AA?$DN?$AA?5?$AA0?$AAx?$AA?$CF?$AAx?$AA?5?$AA?$AN@ 100015b8     sgtl5000codec.obj
 0001:000005fc       ??_C@_1DK@COIECEPA@?$AAD?$AAA?$AAP?$AA_?$AAC?$AAO?$AAE?$AAF?$AA_?$AAW?$AAR?$AA_?$AAB?$AA0?$AA_?$AAL?$AAS?$AAB?$AA?5?$AA?$DN?$AA?5?$AA0?$AAx?$AA?$CF?$AAx?$AA?5?$AA?$AN?$AA?6?$AA?$AA@ 100015fc     sgtl5000codec.obj
 0001:00000638       ??_C@_1DK@CPDBNJON@?$AAD?$AAA?$AAP?$AA_?$AAC?$AAO?$AAE?$AAF?$AA_?$AAW?$AAR?$AA_?$AAB?$AA0?$AA_?$AAM?$AAS?$AAB?$AA?5?$AA?$DN?$AA?5?$AA0?$AAx?$AA?$CF?$AAx?$AA?5?$AA?$AN?$AA?6?$AA?$AA@ 10001638     sgtl5000codec.obj
 0001:00000678       ??_C@_1EC@GPIMAIJG@?$AAD?$AAA?$AAP?$AA_?$AAF?$AAI?$AAL?$AAT?$AAE?$AAR?$AA_?$AAC?$AAO?$AAE?$AAF?$AA_?$AAA?$AAC?$AAC?$AAE?$AAS?$AAS?$AA?5?$AA?$DN?$AA?5?$AA0?$AAx?$AA?$CF?$AAx?$AA?5?$AA?$AN?$AA?6@ 10001678     sgtl5000codec.obj
 0001:000006bc       ??_C@_1DI@JLONNFN@?$AAD?$AAA?$AAP?$AA_?$AAS?$AAG?$AAT?$AAL?$AA_?$AAS?$AAU?$AAR?$AAR?$AAO?$AAU?$AAN?$AAD?$AA?5?$AA?$DN?$AA?5?$AA0?$AAx?$AA?$CF?$AAx?$AA?5?$AA?$AN?$AA?6?$AA?$AA@ 100016bc     sgtl5000codec.obj
 0001:000006f4       ??_C@_1CO@PBLJOJLN@?$AAD?$AAA?$AAP?$AA_?$AAA?$AAU?$AAD?$AAI?$AAO?$AA_?$AAE?$AAQ?$AA?5?$AA?$DN?$AA?5?$AA0?$AAx?$AA?$CF?$AAx?$AA?5?$AA?$AN?$AA?6?$AA?$AA@ 100016f4     sgtl5000codec.obj
 0001:00000728       ??_C@_1EA@CMOGMMAO@?$AAD?$AAA?$AAP?$AA_?$AAB?$AAA?$AAS?$AAS?$AA_?$AAE?$AAN?$AAH?$AAA?$AAN?$AAC?$AAE?$AA_?$AAC?$AAT?$AAR?$AAL?$AA?5?$AA?$DN?$AA?5?$AA0?$AAx?$AA?$CF?$AAx?$AA?5?$AA?$AN?$AA?6?$AA?$AA@ 10001728     sgtl5000codec.obj
 0001:00000768       ??_C@_1DG@INCKILDE@?$AAD?$AAA?$AAP?$AA_?$AAB?$AAA?$AAS?$AAS?$AA_?$AAE?$AAN?$AAH?$AAA?$AAN?$AAC?$AAE?$AA?5?$AA?$DN?$AA?5?$AA0?$AAx?$AA?$CF?$AAx?$AA?5?$AA?$AN?$AA?6?$AA?$AA@ 10001768     sgtl5000codec.obj
 0001:000007a0       ??_C@_1CE@PIMFOJBH@?$AAD?$AAA?$AAP?$AA_?$AAP?$AAE?$AAQ?$AA?5?$AA?$DN?$AA?5?$AA0?$AAx?$AA?$CF?$AAx?$AA?5?$AA?$AN?$AA?6?$AA?$AA@ 100017a0     sgtl5000codec.obj
 0001:000007c4       ??_C@_1CM@FFLLOJIP@?$AAD?$AAA?$AAP?$AA_?$AAC?$AAO?$AAN?$AAT?$AAR?$AAO?$AAL?$AA?5?$AA?$DN?$AA?5?$AA0?$AAx?$AA?$CF?$AAx?$AA?5?$AA?$AN?$AA?6?$AA?$AA@ 100017c4     sgtl5000codec.obj
 0001:000007f0       ??_C@_1DE@MCEIDPPJ@?$AAC?$AAH?$AAI?$AAP?$AA_?$AAS?$AAH?$AAO?$AAR?$AAT?$AA_?$AAC?$AAT?$AAR?$AAL?$AA?5?$AA?$DN?$AA?5?$AA0?$AAx?$AA?$CF?$AAx?$AA?5?$AA?$AN?$AA?6?$AA?$AA@ 100017f0     sgtl5000codec.obj
 0001:00000824       ??_C@_1DE@FMMLNMF@?$AAC?$AAH?$AAI?$AAP?$AA_?$AAA?$AAN?$AAA?$AA_?$AAS?$AAT?$AAA?$AAT?$AAU?$AAS?$AA?5?$AA?$DN?$AA?5?$AA0?$AAx?$AA?$CF?$AAx?$AA?5?$AA?$AN?$AA?6?$AA?$AA@ 10001824     sgtl5000codec.obj
 0001:00000858       ??_C@_1DI@NNPOMNCE@?$AAC?$AAH?$AAI?$AAP?$AA_?$AAC?$AAL?$AAK?$AA_?$AAT?$AAO?$AAP?$AA_?$AAC?$AAT?$AAR?$AAL?$AA?5?$AA?$DN?$AA?5?$AA0?$AAx?$AA?$CF?$AAx?$AA?5?$AA?$AN?$AA?6?$AA?$AA@ 10001858     sgtl5000codec.obj
 0001:00000890       ??_C@_1DA@KKFJADKM@?$AAC?$AAH?$AAI?$AAP?$AA_?$AAP?$AAL?$AAL?$AA_?$AAC?$AAT?$AAR?$AAL?$AA?5?$AA?$DN?$AA?5?$AA0?$AAx?$AA?$CF?$AAx?$AA?5?$AA?$AN?$AA?6?$AA?$AA@ 10001890     sgtl5000codec.obj
 0001:000008c0       ??_C@_1DC@DIMAIPID@?$AAC?$AAH?$AAI?$AAP?$AA_?$AAA?$AAN?$AAA?$AA_?$AAP?$AAO?$AAW?$AAE?$AAR?$AA?5?$AA?$DN?$AA?5?$AA0?$AAx?$AA?$CF?$AAx?$AA?5?$AA?$AN?$AA?6?$AA?$AA@ 100018c0     sgtl5000codec.obj
 0001:000008f4       ??_C@_1DI@BOHMPMFH@?$AAC?$AAH?$AAI?$AAP?$AA_?$AAL?$AAI?$AAN?$AAE?$AA_?$AAO?$AAU?$AAT?$AA_?$AAV?$AAO?$AAL?$AA?5?$AA?$DN?$AA?5?$AA0?$AAx?$AA?$CF?$AAx?$AA?5?$AA?$AN?$AA?6?$AA?$AA@ 100018f4     sgtl5000codec.obj
 0001:0000092c       ??_C@_1DK@LNDNIJNB@?$AAC?$AAH?$AAI?$AAP?$AA_?$AAL?$AAI?$AAN?$AAE?$AA_?$AAO?$AAU?$AAT?$AA_?$AAC?$AAT?$AAR?$AAL?$AA?5?$AA?$DN?$AA?5?$AA0?$AAx?$AA?$CF?$AAx?$AA?5?$AA?$AN?$AA?6?$AA?$AA@ 1000192c     sgtl5000codec.obj
 0001:00000968       ??_C@_1DA@NDHOLOIP@?$AAC?$AAH?$AAI?$AAP?$AA_?$AAM?$AAI?$AAC?$AA_?$AAC?$AAT?$AAR?$AAL?$AA?5?$AA?$DN?$AA?5?$AA0?$AAx?$AA?$CF?$AAx?$AA?5?$AA?$AN?$AA?6?$AA?$AA@ 10001968     sgtl5000codec.obj
 0001:00000998       ??_C@_1DA@DJIOLGAP@?$AAC?$AAH?$AAI?$AAP?$AA_?$AAR?$AAE?$AAF?$AA_?$AAC?$AAT?$AAR?$AAL?$AA?5?$AA?$DN?$AA?5?$AA0?$AAx?$AA?$CF?$AAx?$AA?5?$AA?$AN?$AA?6?$AA?$AA@ 10001998     sgtl5000codec.obj
 0001:000009c8       ??_C@_1DG@FKCBDHPA@?$AAC?$AAH?$AAI?$AAP?$AA_?$AAL?$AAI?$AAN?$AAR?$AAE?$AAG?$AA_?$AAC?$AAT?$AAR?$AAL?$AA?5?$AA?$DN?$AA?5?$AA0?$AAx?$AA?$CF?$AAx?$AA?5?$AA?$AN?$AA?6?$AA?$AA@ 100019c8     sgtl5000codec.obj
 0001:00000a00       ??_C@_1DA@CKBLDIFH@?$AAC?$AAH?$AAI?$AAP?$AA_?$AAA?$AAN?$AAA?$AA_?$AAC?$AAT?$AAR?$AAL?$AA?5?$AA?$DN?$AA?5?$AA0?$AAx?$AA?$CF?$AAx?$AA?5?$AA?$AN?$AA?6?$AA?$AA@ 10001a00     sgtl5000codec.obj
 0001:00000a30       ??_C@_1DG@GFHJKCNJ@?$AAC?$AAH?$AAI?$AAP?$AA_?$AAA?$AAN?$AAA?$AA_?$AAH?$AAP?$AA_?$AAC?$AAT?$AAR?$AAL?$AA?5?$AA?$DN?$AA?5?$AA0?$AAx?$AA?$CF?$AAx?$AA?5?$AA?$AN?$AA?6?$AA?$AA@ 10001a30     sgtl5000codec.obj
 0001:00000a68       ??_C@_1DI@NJFOGCAB@?$AAC?$AAH?$AAI?$AAP?$AA_?$AAA?$AAN?$AAA?$AA_?$AAA?$AAD?$AAC?$AA_?$AAC?$AAT?$AAR?$AAL?$AA?5?$AA?$DN?$AA?5?$AA0?$AAx?$AA?$CF?$AAx?$AA?5?$AA?$AN?$AA?6?$AA?$AA@ 10001a68     sgtl5000codec.obj
 0001:00000aa0       ??_C@_1EA@MEPKMBMN@?$AAC?$AAH?$AAI?$AAP?$AA_?$AAP?$AAA?$AAD?$AA_?$AAS?$AAT?$AAR?$AAE?$AAN?$AAG?$AAT?$AAH?$AA_?$AAA?$AAD?$AAD?$AAR?$AA?$DN?$AA?5?$AA0?$AAx?$AA?$CF?$AAx?$AA?5?$AA?$AN?$AA?6?$AA?$AA@ 10001aa0     sgtl5000codec.obj
 0001:00000ae0       ??_C@_1CO@DHMOBPCF@?$AAC?$AAH?$AAI?$AAP?$AA_?$AAD?$AAA?$AAC?$AA_?$AAV?$AAO?$AAL?$AA?5?$AA?$DN?$AA?5?$AA0?$AAx?$AA?$CF?$AAx?$AA?5?$AA?$AN?$AA?6?$AA?$AA@ 10001ae0     sgtl5000codec.obj
 0001:00000b10       ??_C@_1DG@JCMDDNOC@?$AAC?$AAH?$AAI?$AAP?$AA_?$AAA?$AAD?$AAC?$AAD?$AAA?$AAC?$AA_?$AAC?$AAT?$AAR?$AAL?$AA?5?$AA?$DN?$AA?5?$AA0?$AAx?$AA?$CF?$AAx?$AA?5?$AA?$AN?$AA?6?$AA?$AA@ 10001b10     sgtl5000codec.obj
 0001:00000b48       ??_C@_1DA@PLKNCAA@?$AAC?$AAH?$AAI?$AAP?$AA_?$AAS?$AAS?$AAS?$AA_?$AAC?$AAT?$AAR?$AAL?$AA?5?$AA?$DN?$AA?5?$AA0?$AAx?$AA?$CF?$AAx?$AA?5?$AA?$AN?$AA?6?$AA?$AA@ 10001b48     sgtl5000codec.obj
 0001:00000b78       ??_C@_1DA@HCGNLFOA@?$AAC?$AAH?$AAI?$AAP?$AA_?$AAI?$AA2?$AAS?$AA_?$AAC?$AAT?$AAR?$AAL?$AA?5?$AA?$DN?$AA?5?$AA0?$AAx?$AA?$CF?$AAx?$AA?5?$AA?$AN?$AA?6?$AA?$AA@ 10001b78     sgtl5000codec.obj
 0001:00000ba8       ??_C@_1DA@KNIMEHCE@?$AAC?$AAH?$AAI?$AAP?$AA_?$AAC?$AAL?$AAK?$AA_?$AAC?$AAT?$AAR?$AAL?$AA?5?$AA?$DN?$AA?5?$AA0?$AAx?$AA?$CF?$AAx?$AA?5?$AA?$AN?$AA?6?$AA?$AA@ 10001ba8     sgtl5000codec.obj
 0001:00000bd8       ??_C@_1DC@JIJNFEML@?$AAC?$AAH?$AAI?$AAP?$AA_?$AAD?$AAI?$AAG?$AA_?$AAP?$AAO?$AAW?$AAE?$AAR?$AA?5?$AA?$DN?$AA?5?$AA0?$AAx?$AA?$CF?$AAx?$AA?5?$AA?$AN?$AA?6?$AA?$AA@ 10001bd8     sgtl5000codec.obj
 0001:00000c0c       ??_C@_1CE@BMAENIAL@?$AAC?$AAH?$AAI?$AAP?$AA_?$AAI?$AAD?$AA?5?$AA?$DN?$AA?5?$AA0?$AAx?$AA?$CF?$AAx?$AA?5?$AA?$AN?$AA?6?$AA?$AA@ 10001c0c     sgtl5000codec.obj
 0001:00000c30       ??_C@_1EG@HNGKJHAH@?$AAW?$AAA?$AAV?$AA_?$AAI?$AAo?$AAC?$AAo?$AAn?$AAt?$AAr?$AAo?$AAl?$AA?3?$AA?5?$AAu?$AAn?$AAt?$AAr?$AAu?$AAs?$AAt?$AAe?$AAd?$AA?5?$AAp?$AAr?$AAo?$AAc?$AAe?$AAs?$AAs@ 10001c30     wavedev2_common_topaz_v1:wavemain.obj
 0001:00000c78       ??_7InputDeviceContext@@6B@ 10001c78     wavedev2_common_topaz_v1:hwctxt.obj
 0001:00000c98       ??_7OutputDeviceContext@@6B@ 10001c98     wavedev2_common_topaz_v1:hwctxt.obj
 0001:00000cb8       ??_C@_1IG@IHIMBDHK@?$AA?$FL?$AAE?$AAR?$AAR?$AAO?$AAR?$AA?$FN?$AA?5?$AA?$CC?$AAF?$AAa?$AAi?$AAl?$AAe?$AAd?$AA?5?$AAt?$AAo?$AA?5?$AAi?$AAn?$AAi?$AAt?$AAi?$AAa?$AAl?$AAi?$AAz?$AAe?$AA?5?$AAh?$AAe@ 10001cb8     wavedev2_common_topaz_v1:hwctxt.obj
 0001:00000d40       ??_C@_1GM@MBFOFELI@?$AA?$FL?$AAE?$AAR?$AAR?$AAO?$AAR?$AA?$FN?$AA?5?$AA?$CC?$AAF?$AAa?$AAi?$AAl?$AAe?$AAd?$AA?5?$AAt?$AAo?$AA?5?$AAi?$AAn?$AAi?$AAt?$AAi?$AAa?$AAl?$AAi?$AAz?$AAe?$AA?5?$AAd?$AAi@ 10001d40     wavedev2_common_topaz_v1:hwctxt.obj
 0001:00000db0       ??_C@_1HC@FLCGCADO@?$AA?$FL?$AAE?$AAR?$AAR?$AAO?$AAR?$AA?$FN?$AA?5?$AA?$CC?$AAF?$AAa?$AAi?$AAl?$AAe?$AAd?$AA?5?$AAt?$AAo?$AA?5?$AAi?$AAn?$AAi?$AAt?$AAi?$AAa?$AAl?$AAi?$AAz?$AAe?$AA?5?$AAo?$AAu@ 10001db0     wavedev2_common_topaz_v1:hwctxt.obj
 0001:00000e28       ??_C@_1FE@JMDKDDKE@?$AA?$FL?$AAE?$AAR?$AAR?$AAO?$AAR?$AA?$FN?$AA?5?$AA?$CC?$AAI?$AAn?$AAi?$AAt?$AAi?$AAa?$AAl?$AAi?$AAz?$AAe?$AA?5?$AAA?$AAu?$AAd?$AAi?$AAo?$AA?5?$AAC?$AAo?$AAd?$AAe?$AAc?$AA?5@ 10001e28     wavedev2_common_topaz_v1:hwctxt.obj
 0001:00000e80       ??_C@_1FG@KNAIGBMA@?$AA?$FL?$AAE?$AAR?$AAR?$AAO?$AAR?$AA?$FN?$AA?5?$AA?$CC?$AAM?$AAm?$AAM?$AAa?$AAp?$AAI?$AAo?$AAS?$AAp?$AAa?$AAc?$AAe?$AA?5?$AAf?$AAa?$AAi?$AAl?$AAe?$AAd?$AA?5?$AAf?$AAo?$AAr@ 10001e80     wavedev2_common_topaz_v1:hwctxt.obj
 0001:00000ed8       ??_C@_1FA@IMHNCIEO@?$AA?$FL?$AAE?$AAR?$AAR?$AAO?$AAR?$AA?$FN?$AA?5?$AA?$CC?$AAM?$AAm?$AAM?$AAa?$AAp?$AAI?$AAo?$AAS?$AAp?$AAa?$AAc?$AAe?$AA?5?$AAf?$AAa?$AAi?$AAl?$AAe?$AAd?$AA?5?$AAf?$AAo?$AAr@ 10001ed8     wavedev2_common_topaz_v1:hwctxt.obj
 0001:00000f28       ??_C@_1GE@JLPKGJBM@?$AA?$FL?$AAE?$AAR?$AAR?$AAO?$AAR?$AA?$FN?$AA?5?$AA?$CC?$AAI?$AAn?$AAi?$AAt?$AAO?$AAu?$AAt?$AAp?$AAu?$AAt?$AAD?$AAM?$AAA?$AA?3?$AA?5?$AAS?$AAy?$AAs?$AAi?$AAn?$AAt?$AAr?$AA?5@ 10001f28     wavedev2_common_topaz_v1:hwctxt.obj
 0001:00000f90       ??_C@_1HK@PBBJOECN@?$AA?$FL?$AAE?$AAR?$AAR?$AAO?$AAR?$AA?$FN?$AA?5?$AA?$CC?$AAI?$AAn?$AAi?$AAt?$AAO?$AAu?$AAt?$AAp?$AAu?$AAt?$AAD?$AAM?$AAA?$AA?3?$AA?5?$AAB?$AAU?$AAF?$AAF?$AAE?$AAR?$AA_?$AAB@ 10001f90     wavedev2_common_topaz_v1:hwctxt.obj
 0001:00001010       ??_C@_1HK@HFBMHBPN@?$AA?$FL?$AAE?$AAR?$AAR?$AAO?$AAR?$AA?$FN?$AA?5?$AA?$CC?$AAI?$AAn?$AAi?$AAt?$AAO?$AAu?$AAt?$AAp?$AAu?$AAt?$AAD?$AAM?$AAA?$AA?3?$AA?5?$AAB?$AAU?$AAF?$AAF?$AAE?$AAR?$AA_?$AAA@ 10002010     wavedev2_common_topaz_v1:hwctxt.obj
 0001:00001090       ??_C@_1FO@LLNJHCHH@?$AA?$FL?$AAE?$AAR?$AAR?$AAO?$AAR?$AA?$FN?$AA?5?$AA?$CC?$AAI?$AAn?$AAi?$AAt?$AAO?$AAu?$AAt?$AAp?$AAu?$AAt?$AAD?$AAM?$AAA?$AA?3?$AA?5?$AAI?$AAn?$AAv?$AAa?$AAl?$AAi?$AAd?$AA?5@ 10002090     wavedev2_common_topaz_v1:hwctxt.obj
 0001:000010f0       ??_C@_1GI@DIOKBAMH@?$AA?$FL?$AAE?$AAR?$AAR?$AAO?$AAR?$AA?$FN?$AA?5?$AA?$CC?$AAI?$AAn?$AAi?$AAt?$AAO?$AAu?$AAt?$AAp?$AAu?$AAt?$AAD?$AAM?$AAA?$AA?3?$AA?5?$AAD?$AAD?$AAK?$AAS?$AAd?$AAm?$AAa?$AAA@ 100020f0     wavedev2_common_topaz_v1:hwctxt.obj
 0001:00001158       ??_C@_1GE@CGBHHGFP@?$AA?$FL?$AAE?$AAR?$AAR?$AAO?$AAR?$AA?$FN?$AA?5?$AA?$CC?$AAI?$AAn?$AAi?$AAt?$AAO?$AAu?$AAt?$AAp?$AAu?$AAt?$AAD?$AAM?$AAA?$AA?3?$AA?5?$AAD?$AAD?$AAK?$AAS?$AAd?$AAm?$AAa?$AAO@ 10002158     wavedev2_common_topaz_v1:hwctxt.obj
 0001:000011c0       ??_C@_1HK@EHPEHBIH@?$AA?$FL?$AAE?$AAR?$AAR?$AAO?$AAR?$AA?$FN?$AA?5?$AA?$CC?$AAI?$AAn?$AAi?$AAt?$AAO?$AAu?$AAt?$AAp?$AAu?$AAt?$AAD?$AAM?$AAA?$AA?3?$AA?5?$AAD?$AAM?$AAA?$AA?5?$AAb?$AAu?$AAf?$AAf@ 100021c0     wavedev2_common_topaz_v1:hwctxt.obj
 0001:00001240       ??_C@_1GC@OFELANKM@?$AA?$FL?$AAE?$AAR?$AAR?$AAO?$AAR?$AA?$FN?$AA?5?$AA?$CC?$AAI?$AAn?$AAi?$AAt?$AAI?$AAn?$AAp?$AAu?$AAt?$AAD?$AAM?$AAA?$AA?3?$AA?5?$AAS?$AAy?$AAs?$AAi?$AAn?$AAt?$AAr?$AA?5?$AAr@ 10002240     wavedev2_common_topaz_v1:hwctxt.obj
 0001:000012a8       ??_C@_1HI@PGFDCGBG@?$AA?$FL?$AAE?$AAR?$AAR?$AAO?$AAR?$AA?$FN?$AA?5?$AA?$CC?$AAI?$AAn?$AAi?$AAt?$AAI?$AAn?$AAp?$AAu?$AAt?$AAD?$AAM?$AAA?$AA?3?$AA?5?$AAB?$AAU?$AAF?$AAF?$AAE?$AAR?$AA_?$AAB?$AA?5@ 100022a8     wavedev2_common_topaz_v1:hwctxt.obj
 0001:00001320       ??_C@_1HI@HCFGLDMG@?$AA?$FL?$AAE?$AAR?$AAR?$AAO?$AAR?$AA?$FN?$AA?5?$AA?$CC?$AAI?$AAn?$AAi?$AAt?$AAI?$AAn?$AAp?$AAu?$AAt?$AAD?$AAM?$AAA?$AA?3?$AA?5?$AAB?$AAU?$AAF?$AAF?$AAE?$AAR?$AA_?$AAA?$AA?5@ 10002320     wavedev2_common_topaz_v1:hwctxt.obj
 0001:00001398       ??_C@_1FM@OIAIFOP@?$AA?$FL?$AAE?$AAR?$AAR?$AAO?$AAR?$AA?$FN?$AA?5?$AA?$CC?$AAI?$AAn?$AAi?$AAt?$AAI?$AAn?$AAp?$AAu?$AAt?$AAD?$AAM?$AAA?$AA?3?$AA?5?$AAI?$AAn?$AAv?$AAa?$AAl?$AAi?$AAd?$AA?5?$AAs@ 10002398     wavedev2_common_topaz_v1:hwctxt.obj
 0001:000013f8       ??_C@_1GG@CACFPOGD@?$AA?$FL?$AAE?$AAR?$AAR?$AAO?$AAR?$AA?$FN?$AA?5?$AA?$CC?$AAI?$AAn?$AAi?$AAt?$AAI?$AAn?$AAp?$AAu?$AAt?$AAD?$AAM?$AAA?$AA?3?$AA?5?$AAD?$AAD?$AAK?$AAS?$AAd?$AAm?$AAa?$AAA?$AAl@ 100023f8     wavedev2_common_topaz_v1:hwctxt.obj
 0001:00001460       ??_C@_1GC@FIKGBCOP@?$AA?$FL?$AAE?$AAR?$AAR?$AAO?$AAR?$AA?$FN?$AA?5?$AA?$CC?$AAI?$AAn?$AAi?$AAt?$AAI?$AAn?$AAp?$AAu?$AAt?$AAD?$AAM?$AAA?$AA?3?$AA?5?$AAD?$AAD?$AAK?$AAS?$AAd?$AAm?$AAa?$AAO?$AAp@ 10002460     wavedev2_common_topaz_v1:hwctxt.obj
 0001:000014c8       ??_C@_1HI@EALOLDLM@?$AA?$FL?$AAE?$AAR?$AAR?$AAO?$AAR?$AA?$FN?$AA?5?$AA?$CC?$AAI?$AAn?$AAi?$AAt?$AAI?$AAn?$AAp?$AAu?$AAt?$AAD?$AAM?$AAA?$AA?3?$AA?5?$AAD?$AAM?$AAA?$AA?5?$AAb?$AAu?$AAf?$AAf?$AAe@ 100024c8     wavedev2_common_topaz_v1:hwctxt.obj
 0001:00001540       ??_C@_1BI@BHLBGEOK@?$AAP?$AAr?$AAi?$AAo?$AAr?$AAi?$AAt?$AAy?$AA2?$AA5?$AA6?$AA?$AA@ 10002540     wavedev2_common_topaz_v1:hwctxt.obj
 0001:00001558       ??_C@_1IA@LBNHHCMD@?$AA?$FL?$AAE?$AAR?$AAR?$AAO?$AAR?$AA?$FN?$AA?5?$AA?$CC?$AAI?$AAn?$AAi?$AAt?$AAH?$AAP?$AAD?$AAe?$AAt?$AAe?$AAc?$AAt?$AAI?$AAn?$AAt?$AAe?$AAr?$AAr?$AAu?$AAp?$AAt?$AAT?$AAh@ 10002558     wavedev2_common_topaz_v1:hwctxt.obj
 0001:000015d8       ??_C@_1KK@JEOCOOEC@?$AA?$FL?$AAE?$AAR?$AAR?$AAO?$AAR?$AA?$FN?$AA?5?$AA?$CC?$AAU?$AAn?$AAa?$AAb?$AAl?$AAe?$AA?5?$AAt?$AAo?$AA?5?$AAc?$AAr?$AAe?$AAa?$AAt?$AAe?$AA?5?$AAa?$AAu?$AAd?$AAi?$AAo?$AA?5@ 100025d8     wavedev2_common_topaz_v1:hwctxt.obj
 0001:00001688       ??_C@_1FE@OGEABEJC@?$AA?$FL?$AAE?$AAR?$AAR?$AAO?$AAR?$AA?$FN?$AA?5?$AA?$CC?$AAU?$AAn?$AAa?$AAb?$AAl?$AAe?$AA?5?$AAt?$AAo?$AA?5?$AAc?$AAr?$AAe?$AAa?$AAt?$AAe?$AA?5?$AAd?$AAe?$AAl?$AAa?$AAy?$AA?5@ 10002688     wavedev2_common_topaz_v1:hwctxt.obj
 0001:000016e0       ??_C@_1JA@KMMGDDKB@?$AA?$FL?$AAE?$AAR?$AAR?$AAO?$AAR?$AA?$FN?$AA?5?$AA?$CC?$AAS?$AAt?$AAa?$AAr?$AAt?$AAO?$AAu?$AAt?$AAp?$AAu?$AAt?$AAD?$AAM?$AAA?$AA?3?$AA?5?$AAU?$AAn?$AAa?$AAb?$AAl?$AAe?$AA?5@ 100026e0     wavedev2_common_topaz_v1:hwctxt.obj
 0001:00001770       ??_C@_1IO@PIJKJFCE@?$AA?$FL?$AAE?$AAR?$AAR?$AAO?$AAR?$AA?$FN?$AA?5?$AA?$CC?$AAS?$AAt?$AAa?$AAr?$AAt?$AAI?$AAn?$AAp?$AAu?$AAt?$AAD?$AAM?$AAA?$AA?3?$AA?5?$AAU?$AAn?$AAa?$AAb?$AAl?$AAe?$AA?5?$AAt@ 10002770     wavedev2_common_topaz_v1:hwctxt.obj
 0001:00001800       ??_C@_1IC@JIBANBOM@?$AAS?$AAt?$AAa?$AAr?$AAt?$AAI?$AAn?$AAp?$AAu?$AAt?$AAD?$AAM?$AAA?$AA?3?$AA?5?$AAR?$AAe?$AAc?$AAo?$AAr?$AAd?$AAi?$AAn?$AAg?$AA?5?$AAc?$AAa?$AAn?$AA?5?$AAn?$AAo?$AAt@ 10002800     wavedev2_common_topaz_v1:hwctxt.obj
 0001:00001888       ??_C@_1HC@IDPKCCMA@?$AA?$FL?$AAE?$AAR?$AAR?$AAO?$AAR?$AA?$FN?$AA?5?$AA?$CC?$AAE?$AAr?$AAr?$AAo?$AAr?$AA?5?$AAf?$AAl?$AAa?$AAg?$AA?5?$AAs?$AAe?$AAt?$AA?5?$AAi?$AAn?$AA?5?$AAo?$AAu?$AAt?$AAp?$AAu@ 10002888     wavedev2_common_topaz_v1:hwctxt.obj
 0001:00001900       ??_C@_1HC@EKOFCKHP@?$AA?$FL?$AAE?$AAR?$AAR?$AAO?$AAR?$AA?$FN?$AA?5?$AA?$CC?$AAE?$AAr?$AAr?$AAo?$AAr?$AA?5?$AAf?$AAl?$AAa?$AAg?$AA?5?$AAs?$AAe?$AAt?$AA?5?$AAi?$AAn?$AA?5?$AAo?$AAu?$AAt?$AAp?$AAu@ 10002900     wavedev2_common_topaz_v1:hwctxt.obj
 0001:00001978       ??_C@_1GI@JJHJOGE@?$AA?$FL?$AAE?$AAR?$AAR?$AAO?$AAR?$AA?$FN?$AA?5?$AA?$CC?$AAC?$AAo?$AAu?$AAl?$AAd?$AA?5?$AAn?$AAo?$AAt?$AA?5?$AAr?$AAe?$AAt?$AAr?$AAi?$AAe?$AAv?$AAe?$AA?5?$AAo?$AAu?$AAt?$AAp@ 10002978     wavedev2_common_topaz_v1:hwctxt.obj
 0001:000019e0       ??_C@_1CE@DCGOLNHM@?$AAS?$AAS?$AAI?$AA?5?$AAT?$AAX?$AA?5?$AAu?$AAn?$AAd?$AAe?$AAr?$AAr?$AAu?$AAn?$AA?$AN?$AA?6?$AA?$AA@ 100029e0     wavedev2_common_topaz_v1:hwctxt.obj
 0001:00001a08       ??_C@_1FK@LCONGMCG@?$AA?$FL?$AAE?$AAR?$AAR?$AAO?$AAR?$AA?$FN?$AA?5?$AA?$CC?$AAE?$AAr?$AAr?$AAo?$AAr?$AA?5?$AAf?$AAl?$AAa?$AAg?$AA?5?$AAs?$AAe?$AAt?$AA?5?$AAi?$AAn?$AA?5?$AAi?$AAn?$AAp?$AAu?$AAt@ 10002a08     wavedev2_common_topaz_v1:hwctxt.obj
 0001:00001a68       ??_C@_1HA@NFNHLKKL@?$AA?$FL?$AAE?$AAR?$AAR?$AAO?$AAR?$AA?$FN?$AA?5?$AA?$CC?$AAE?$AAr?$AAr?$AAo?$AAr?$AA?5?$AAf?$AAl?$AAa?$AAg?$AA?5?$AAs?$AAe?$AAt?$AA?5?$AAi?$AAn?$AA?5?$AAi?$AAn?$AAp?$AAu?$AAt@ 10002a68     wavedev2_common_topaz_v1:hwctxt.obj
 0001:00001ad8       ??_C@_1GG@LDFKJMLF@?$AA?$FL?$AAE?$AAR?$AAR?$AAO?$AAR?$AA?$FN?$AA?5?$AA?$CC?$AAC?$AAo?$AAu?$AAl?$AAd?$AA?5?$AAn?$AAo?$AAt?$AA?5?$AAr?$AAe?$AAt?$AAr?$AAi?$AAe?$AAv?$AAe?$AA?5?$AAi?$AAn?$AAp?$AAu@ 10002ad8     wavedev2_common_topaz_v1:hwctxt.obj
 0001:00001b40       ??_C@_1CC@IBAPKJHP@?$AAS?$AAS?$AAI?$AA?5?$AAR?$AAX?$AA?5?$AAo?$AAv?$AAe?$AAr?$AAr?$AAu?$AAn?$AA?$AN?$AA?6?$AA?$AA@ 10002b40     wavedev2_common_topaz_v1:hwctxt.obj
 0001:00001b64       ??_C@_1DC@CBAPFGDJ@?$AAS?$AAk?$AAi?$AAp?$AA?5?$AAd?$AAi?$AAs?$AAa?$AAb?$AAl?$AAi?$AAn?$AAg?$AA?5?$AAt?$AAh?$AAe?$AA?5?$AAA?$AAD?$AAC?$AA?$AN?$AA?6?$AA?$AA@ 10002b64     wavedev2_common_topaz_v1:hwctxt.obj
 0001:00001b98       ??_C@_1DC@FPIFOKGN@?$AAS?$AAk?$AAi?$AAp?$AA?5?$AAd?$AAi?$AAs?$AAa?$AAb?$AAl?$AAi?$AAn?$AAg?$AA?5?$AAt?$AAh?$AAe?$AA?5?$AAD?$AAA?$AAC?$AA?$AN?$AA?6?$AA?$AA@ 10002b98     wavedev2_common_topaz_v1:hwctxt.obj
 0001:00001bd0       ??_C@_1EI@IJIJICDH@?$AAW?$AAA?$AAV?$AAE?$AA?3?$AA?5?$AAU?$AAn?$AAk?$AAn?$AAo?$AAw?$AAn?$AA?5?$AAI?$AAO?$AAC?$AAT?$AAL?$AA_?$AAx?$AAx?$AAx?$AA?$CI?$AA0?$AAx?$AA?$CF?$AA0?$AA?4?$AA8?$AAX?$AA?$CJ@ 10002bd0     wavedev2_common_topaz_v1:hwctxt.obj
 0001:00001c18       ??_C@_1FE@BFNEOFLI@?$AAW?$AAA?$AAV?$AAE?$AA?3?$AA?5?$AAI?$AAO?$AAC?$AAT?$AAL?$AA_?$AAP?$AAO?$AAW?$AAE?$AAR?$AA_?$AAG?$AAE?$AAT?$AA?5?$AA?9?$AA?9?$AA?5?$AAn?$AAo?$AAt?$AA?5?$AAs?$AAu?$AAp@ 10002c18     wavedev2_common_topaz_v1:hwctxt.obj
 0001:00001c70       ??_C@_1FG@NBOCOKEO@?$AAW?$AAA?$AAV?$AAE?$AA?3?$AA?5?$AAI?$AAO?$AAC?$AAT?$AAL?$AA_?$AAP?$AAO?$AAW?$AAE?$AAR?$AA_?$AAS?$AAE?$AAT?$AA?5?$AAi?$AAn?$AAv?$AAa?$AAl?$AAi?$AAd?$AA?5?$AAp?$AAa@ 10002c70     wavedev2_common_topaz_v1:hwctxt.obj
 0001:00001cc8       ??_C@_1FK@IMHALGMP@?$AAW?$AAA?$AAV?$AAE?$AA?3?$AA?5?$AAI?$AAO?$AAC?$AAT?$AAL?$AA_?$AAP?$AAO?$AAW?$AAE?$AAR?$AA_?$AAS?$AAE?$AAT?$AA?5?$AAi?$AAn?$AAv?$AAa?$AAl?$AAi?$AAd?$AA?5?$AAp?$AAo@ 10002cc8     wavedev2_common_topaz_v1:hwctxt.obj
 0001:00001d24       ??_C@_1DM@LLGCMHAC@?$AAW?$AAA?$AAV?$AAE?$AA?3?$AA?5?$AAI?$AAO?$AAC?$AAT?$AAL?$AA_?$AAP?$AAO?$AAW?$AAE?$AAR?$AA_?$AAS?$AAE?$AAT?$AA?5?$AA?$DN?$AA?5?$AA?$CF?$AAd?$AA?4?$AA?$AN?$AA?6?$AA?$AA@ 10002d24     wavedev2_common_topaz_v1:hwctxt.obj
 0001:00001d60       ??_C@_1FK@JAMKGCEM@?$AAW?$AAA?$AAV?$AAE?$AA?3?$AA?5?$AAI?$AAO?$AAC?$AAT?$AAL?$AA_?$AAP?$AAO?$AAW?$AAE?$AAR?$AA_?$AAQ?$AAU?$AAE?$AAR?$AAY?$AA?5?$AAi?$AAn?$AAv?$AAa?$AAl?$AAi?$AAd?$AA?5@ 10002d60     wavedev2_common_topaz_v1:hwctxt.obj
 0001:00001dc0       ??_C@_1FO@JFNJOLNA@?$AAW?$AAA?$AAV?$AAE?$AA?3?$AA?5?$AAI?$AAO?$AAC?$AAT?$AAL?$AA_?$AAP?$AAO?$AAW?$AAE?$AAR?$AA_?$AAQ?$AAU?$AAE?$AAR?$AAY?$AA?5?$AAi?$AAn?$AAv?$AAa?$AAl?$AAi?$AAd?$AA?5@ 10002dc0     wavedev2_common_topaz_v1:hwctxt.obj
 0001:00001e20       ??_C@_1DO@CJNFJIKM@?$AAW?$AAA?$AAV?$AAE?$AA?3?$AA?5?$AAI?$AAO?$AAC?$AAT?$AAL?$AA_?$AAP?$AAO?$AAW?$AAE?$AAR?$AA_?$AAQ?$AAU?$AAE?$AAR?$AAY?$AA?5?$AA?$DN?$AA?5?$AA?$CF?$AAd?$AA?$AN?$AA?6?$AA?$AA@ 10002e20     wavedev2_common_topaz_v1:hwctxt.obj
 0001:00001e60       ??_C@_1DG@EDLBLBEC@?$AAW?$AAA?$AAV?$AAE?$AA?3?$AA?5?$AAI?$AAn?$AAv?$AAa?$AAl?$AAi?$AAd?$AA?5?$AAp?$AAa?$AAr?$AAa?$AAm?$AAe?$AAt?$AAe?$AAr?$AA?4?$AA?$AN?$AA?6?$AA?$AA@ 10002e60     wavedev2_common_topaz_v1:hwctxt.obj
 0001:00001e98       ??_C@_1FA@GFIEJBEN@?$AAW?$AAA?$AAV?$AAE?$AA?3?$AA?5?$AAI?$AAO?$AAC?$AAT?$AAL?$AA_?$AAP?$AAO?$AAW?$AAE?$AAR?$AA_?$AAC?$AAA?$AAP?$AAA?$AAB?$AAI?$AAL?$AAI?$AAT?$AAI?$AAE?$AAS?$AA?5?$AA?$DN@ 10002e98     wavedev2_common_topaz_v1:hwctxt.obj
 0001:00001ee8       ??_C@_1HA@NNADDFFI@?$AAC?$AAa?$AAn?$AA?5?$AAn?$AAo?$AAt?$AA?5?$AAc?$AAh?$AAa?$AAn?$AAg?$AAe?$AA?5?$AAi?$AAn?$AAp?$AAu?$AAt?$AA?5?$AAs?$AAo?$AAu?$AAr?$AAc?$AAe?$AA?5?$AAw?$AAh?$AAe?$AAn@ 10002ee8     wavedev2_common_topaz_v1:hwctxt.obj
 0001:00001f58       ??_C@_1FC@MGAHJMFE@?$AAS?$AAe?$AAt?$AAC?$AAo?$AAd?$AAe?$AAc?$AAL?$AAo?$AAo?$AAp?$AAb?$AAa?$AAc?$AAk?$AA?3?$AA?5?$AAR?$AAe?$AAc?$AAo?$AAr?$AAd?$AAi?$AAn?$AAg?$AA?5?$AAi?$AAs?$AA?5?$AAr@ 10002f58     wavedev2_common_topaz_v1:hwctxt.obj
 0001:00001fb0       ??_C@_1FA@LMNDEPJO@?$AAS?$AAe?$AAt?$AAC?$AAo?$AAd?$AAe?$AAc?$AAL?$AAo?$AAo?$AAp?$AAb?$AAa?$AAc?$AAk?$AA?3?$AA?5?$AAP?$AAl?$AAa?$AAy?$AAb?$AAa?$AAc?$AAk?$AA?5?$AAi?$AAs?$AA?5?$AAr?$AAu@ 10002fb0     wavedev2_common_topaz_v1:hwctxt.obj
 0001:00002000       ??_7DeviceContext@@6B@     10003000     wavedev2_common_topaz_v1:devctxt.obj
 0001:00002040       ??_7InputStreamContext@@6B@ 10003040     wavedev2_common_topaz_v1:devctxt.obj
 0001:00002088       ??_7WaveStreamContext@@6B@ 10003088     wavedev2_common_topaz_v1:devctxt.obj
 0001:000020cc       ??_7CMidiStream@@6B@       100030cc     wavedev2_common_topaz_v1:devctxt.obj
 0001:00002108       ??_7OutputStreamContext16bitM8@@6B@ 10003108     wavedev2_common_topaz_v1:devctxt.obj
 0001:00002150       ??_7OutputStreamContext16bitS8@@6B@ 10003150     wavedev2_common_topaz_v1:devctxt.obj
 0001:00002198       ??_7OutputStreamContext16bitM16@@6B@ 10003198     wavedev2_common_topaz_v1:devctxt.obj
 0001:000021e0       ??_7OutputStreamContext16bitS16@@6B@ 100031e0     wavedev2_common_topaz_v1:devctxt.obj
 0001:00002228       ??_7OutputStreamContext24bitM8@@6B@ 10003228     wavedev2_common_topaz_v1:devctxt.obj
 0001:00002270       ??_7OutputStreamContext24bitS8@@6B@ 10003270     wavedev2_common_topaz_v1:devctxt.obj
 0001:000022b8       ??_7OutputStreamContext24bitM16@@6B@ 100032b8     wavedev2_common_topaz_v1:devctxt.obj
 0001:00002300       ??_7OutputStreamContext24bitS16@@6B@ 10003300     wavedev2_common_topaz_v1:devctxt.obj
 0001:00002348       ??_7OutputStreamContext24bitS24@@6B@ 10003348     wavedev2_common_topaz_v1:devctxt.obj
 0001:00002390       ??_7OutputStreamContext@@6B@ 10003390     wavedev2_common_topaz_v1:devctxt.obj
 0001:00002578       ??_7StreamContext@@6B@     10003578     wavedev2_common_topaz_v1:strmctxt.obj
 0001:000025b8       ??_C@_1GI@EBFCCJC@?$AAE?$AAX?$AAC?$AAE?$AAP?$AAT?$AAI?$AAO?$AAN?$AA?5?$AAI?$AAN?$AA?5?$AAI?$AAS?$AAT?$AA?5?$AAf?$AAo?$AAr?$AA?5?$AAs?$AAt?$AAr?$AAe?$AAa?$AAm?$AA?5?$AA0?$AAx?$AA?$CF?$AAx@ 100035b8     wavedev2_common_topaz_v1:strmctxt.obj
 0001:00002620       ??_C@_1BC@JBIMOOCB@?$AAP?$AAl?$AAa?$AAy?$AAb?$AAa?$AAc?$AAk?$AA?$AA@ 10003620     wavedev2_common_topaz_v1:mixerdrv.obj
 0001:00002634       ??_C@_1BA@EEOGCIBB@?$AAL?$AAi?$AAn?$AAe?$AA?5?$AAI?$AAn?$AA?$AA@ 10003634     wavedev2_common_topaz_v1:mixerdrv.obj
 0001:00002644       ??_C@_1BG@OGJPAHBK@?$AAM?$AAi?$AAc?$AAr?$AAo?$AAp?$AAh?$AAo?$AAn?$AAe?$AA?$AA@ 10003644     wavedev2_common_topaz_v1:mixerdrv.obj
 0001:0000265c       ??_C@_1CE@BJPEGCKG@?$AAR?$AAe?$AAc?$AAo?$AAr?$AAd?$AAi?$AAn?$AAg?$AA?5?$AAC?$AAo?$AAn?$AAt?$AAr?$AAo?$AAl?$AA?$AA@ 1000365c     wavedev2_common_topaz_v1:mixerdrv.obj
 0001:00002680       ??_C@_1CA@KOFAABPH@?$AAR?$AAe?$AAc?$AAo?$AAr?$AAd?$AAi?$AAn?$AAg?$AA?5?$AAC?$AAo?$AAn?$AAt?$AAr?$AA?$AA@ 10003680     wavedev2_common_topaz_v1:mixerdrv.obj
 0001:000026a0       ??_C@_1CC@OALPFLIM@?$AAP?$AAl?$AAa?$AAy?$AAb?$AAa?$AAc?$AAk?$AA?5?$AAC?$AAo?$AAn?$AAt?$AAr?$AAo?$AAl?$AA?$AA@ 100036a0     wavedev2_common_topaz_v1:mixerdrv.obj
 0001:000026c4       ??_C@_1BO@OJJBHHKI@?$AAP?$AAl?$AAa?$AAy?$AAb?$AAa?$AAc?$AAk?$AA?5?$AAC?$AAo?$AAn?$AAt?$AAr?$AA?$AA@ 100036c4     wavedev2_common_topaz_v1:mixerdrv.obj
 0001:000026e8       ??_C@_1EG@GKAFBHEE@?$AAM?$AAI?$AAX?$AAE?$AAR?$AAC?$AAO?$AAN?$AAT?$AAR?$AAO?$AAL?$AA_?$AAC?$AAO?$AAN?$AAT?$AAR?$AAO?$AAL?$AAT?$AAY?$AAP?$AAE?$AA_?$AAM?$AAI?$AAL?$AAL?$AAI?$AAT?$AAI@ 100036e8     wavedev2_common_topaz_v1:mixerdrv.obj
 0001:00002730       ??_C@_1EG@KGPLLMHC@?$AAM?$AAI?$AAX?$AAE?$AAR?$AAC?$AAO?$AAN?$AAT?$AAR?$AAO?$AAL?$AA_?$AAC?$AAO?$AAN?$AAT?$AAR?$AAO?$AAL?$AAT?$AAY?$AAP?$AAE?$AA_?$AAM?$AAI?$AAC?$AAR?$AAO?$AAT?$AAI@ 10003730     wavedev2_common_topaz_v1:mixerdrv.obj
 0001:00002778       ??_C@_1EG@MHHEILGF@?$AAM?$AAI?$AAX?$AAE?$AAR?$AAC?$AAO?$AAN?$AAT?$AAR?$AAO?$AAL?$AA_?$AAC?$AAO?$AAN?$AAT?$AAR?$AAO?$AAL?$AAT?$AAY?$AAP?$AAE?$AA_?$AAS?$AAT?$AAE?$AAR?$AAE?$AAO?$AAE@ 10003778     wavedev2_common_topaz_v1:mixerdrv.obj
 0001:000027c0       ??_C@_1DO@MOGMEDOD@?$AAM?$AAI?$AAX?$AAE?$AAR?$AAC?$AAO?$AAN?$AAT?$AAR?$AAO?$AAL?$AA_?$AAC?$AAO?$AAN?$AAT?$AAR?$AAO?$AAL?$AAT?$AAY?$AAP?$AAE?$AA_?$AAO?$AAN?$AAO?$AAF?$AAF?$AA?$AA@ 100037c0     wavedev2_common_topaz_v1:mixerdrv.obj
 0001:00002800       ??_C@_1DM@DCLFABPP@?$AAM?$AAI?$AAX?$AAE?$AAR?$AAC?$AAO?$AAN?$AAT?$AAR?$AAO?$AAL?$AA_?$AAC?$AAO?$AAN?$AAT?$AAR?$AAO?$AAL?$AAT?$AAY?$AAP?$AAE?$AA_?$AAM?$AAU?$AAT?$AAE?$AA?$AA@ 10003800     wavedev2_common_topaz_v1:mixerdrv.obj
 0001:0000283c       ??_C@_1DM@BCDOONIF@?$AAM?$AAI?$AAX?$AAE?$AAR?$AAC?$AAO?$AAN?$AAT?$AAR?$AAO?$AAL?$AA_?$AAC?$AAO?$AAN?$AAT?$AAR?$AAO?$AAL?$AAT?$AAY?$AAP?$AAE?$AA_?$AAM?$AAO?$AAN?$AAO?$AA?$AA@ 1000383c     wavedev2_common_topaz_v1:mixerdrv.obj
 0001:00002878       ??_C@_1EE@FIBKNKLH@?$AAM?$AAI?$AAX?$AAE?$AAR?$AAC?$AAO?$AAN?$AAT?$AAR?$AAO?$AAL?$AA_?$AAC?$AAO?$AAN?$AAT?$AAR?$AAO?$AAL?$AAT?$AAY?$AAP?$AAE?$AA_?$AAL?$AAO?$AAU?$AAD?$AAN?$AAE?$AAS@ 10003878     wavedev2_common_topaz_v1:mixerdrv.obj
 0001:000028c0       ??_C@_1EA@ONOCHFEP@?$AAM?$AAI?$AAX?$AAE?$AAR?$AAC?$AAO?$AAN?$AAT?$AAR?$AAO?$AAL?$AA_?$AAC?$AAO?$AAN?$AAT?$AAR?$AAO?$AAL?$AAT?$AAY?$AAP?$AAE?$AA_?$AAB?$AAU?$AAT?$AAT?$AAO?$AAN?$AA?$AA@ 100038c0     wavedev2_common_topaz_v1:mixerdrv.obj
 0001:00002900       ??_C@_1EC@LBKFNEJB@?$AAM?$AAI?$AAX?$AAE?$AAR?$AAC?$AAO?$AAN?$AAT?$AAR?$AAO?$AAL?$AA_?$AAC?$AAO?$AAN?$AAT?$AAR?$AAO?$AAL?$AAT?$AAY?$AAP?$AAE?$AA_?$AAB?$AAO?$AAO?$AAL?$AAE?$AAA?$AAN@ 10003900     wavedev2_common_topaz_v1:mixerdrv.obj
 0001:00002948       ??_C@_1EA@JCFBIPAK@?$AAM?$AAI?$AAX?$AAE?$AAR?$AAC?$AAO?$AAN?$AAT?$AAR?$AAO?$AAL?$AA_?$AAC?$AAO?$AAN?$AAT?$AAR?$AAO?$AAL?$AAT?$AAY?$AAP?$AAE?$AA_?$AAS?$AAL?$AAI?$AAD?$AAE?$AAR?$AA?$AA@ 10003948     wavedev2_common_topaz_v1:mixerdrv.obj
 0001:00002988       ??_C@_1EG@BEPOGKNO@?$AAM?$AAI?$AAX?$AAE?$AAR?$AAC?$AAO?$AAN?$AAT?$AAR?$AAO?$AAL?$AA_?$AAC?$AAO?$AAN?$AAT?$AAR?$AAO?$AAL?$AAT?$AAY?$AAP?$AAE?$AA_?$AAQ?$AAS?$AAO?$AAU?$AAN?$AAD?$AAP@ 10003988     wavedev2_common_topaz_v1:mixerdrv.obj
 0001:000029d0       ??_C@_1DK@HNKLKPNJ@?$AAM?$AAI?$AAX?$AAE?$AAR?$AAC?$AAO?$AAN?$AAT?$AAR?$AAO?$AAL?$AA_?$AAC?$AAO?$AAN?$AAT?$AAR?$AAO?$AAL?$AAT?$AAY?$AAP?$AAE?$AA_?$AAP?$AAA?$AAN?$AA?$AA@ 100039d0     wavedev2_common_topaz_v1:mixerdrv.obj
 0001:00002a10       ??_C@_1EE@PPIBPMLH@?$AAM?$AAI?$AAX?$AAE?$AAR?$AAC?$AAO?$AAN?$AAT?$AAR?$AAO?$AAL?$AA_?$AAC?$AAO?$AAN?$AAT?$AAR?$AAO?$AAL?$AAT?$AAY?$AAP?$AAE?$AA_?$AAU?$AAN?$AAS?$AAI?$AAG?$AAN?$AAE@ 10003a10     wavedev2_common_topaz_v1:mixerdrv.obj
 0001:00002a58       ??_C@_1EA@PAIJNMCC@?$AAM?$AAI?$AAX?$AAE?$AAR?$AAC?$AAO?$AAN?$AAT?$AAR?$AAO?$AAL?$AA_?$AAC?$AAO?$AAN?$AAT?$AAR?$AAO?$AAL?$AAT?$AAY?$AAP?$AAE?$AA_?$AAS?$AAI?$AAG?$AAN?$AAE?$AAD?$AA?$AA@ 10003a58     wavedev2_common_topaz_v1:mixerdrv.obj
 0001:00002a98       ??_C@_1EC@KPFLKHEG@?$AAM?$AAI?$AAX?$AAE?$AAR?$AAC?$AAO?$AAN?$AAT?$AAR?$AAO?$AAL?$AA_?$AAC?$AAO?$AAN?$AAT?$AAR?$AAO?$AAL?$AAT?$AAY?$AAP?$AAE?$AA_?$AAP?$AAE?$AAR?$AAC?$AAE?$AAN?$AAT@ 10003a98     wavedev2_common_topaz_v1:mixerdrv.obj
 0001:00002ae0       ??_C@_1EE@FDJLOIGD@?$AAM?$AAI?$AAX?$AAE?$AAR?$AAC?$AAO?$AAN?$AAT?$AAR?$AAO?$AAL?$AA_?$AAC?$AAO?$AAN?$AAT?$AAR?$AAO?$AAL?$AAT?$AAY?$AAP?$AAE?$AA_?$AAD?$AAE?$AAC?$AAI?$AAB?$AAE?$AAL@ 10003ae0     wavedev2_common_topaz_v1:mixerdrv.obj
 0001:00002b28       ??_C@_1EO@CIONLEIK@?$AAM?$AAI?$AAX?$AAE?$AAR?$AAC?$AAO?$AAN?$AAT?$AAR?$AAO?$AAL?$AA_?$AAC?$AAO?$AAN?$AAT?$AAR?$AAO?$AAL?$AAT?$AAY?$AAP?$AAE?$AA_?$AAU?$AAN?$AAS?$AAI?$AAG?$AAN?$AAE@ 10003b28     wavedev2_common_topaz_v1:mixerdrv.obj
 0001:00002b78       ??_C@_1EK@KIDDBONI@?$AAM?$AAI?$AAX?$AAE?$AAR?$AAC?$AAO?$AAN?$AAT?$AAR?$AAO?$AAL?$AA_?$AAC?$AAO?$AAN?$AAT?$AAR?$AAO?$AAL?$AAT?$AAY?$AAP?$AAE?$AA_?$AAS?$AAI?$AAG?$AAN?$AAE?$AAD?$AAM@ 10003b78     wavedev2_common_topaz_v1:mixerdrv.obj
 0001:00002bc8       ??_C@_1EG@EBKFDDEH@?$AAM?$AAI?$AAX?$AAE?$AAR?$AAC?$AAO?$AAN?$AAT?$AAR?$AAO?$AAL?$AA_?$AAC?$AAO?$AAN?$AAT?$AAR?$AAO?$AAL?$AAT?$AAY?$AAP?$AAE?$AA_?$AAP?$AAE?$AAA?$AAK?$AAM?$AAE?$AAT@ 10003bc8     wavedev2_common_topaz_v1:mixerdrv.obj
 0001:00002c10       ??_C@_1EM@DKIPIFCO@?$AAM?$AAI?$AAX?$AAE?$AAR?$AAC?$AAO?$AAN?$AAT?$AAR?$AAO?$AAL?$AA_?$AAC?$AAO?$AAN?$AAT?$AAR?$AAO?$AAL?$AAT?$AAY?$AAP?$AAE?$AA_?$AAB?$AAO?$AAO?$AAL?$AAE?$AAA?$AAN@ 10003c10     wavedev2_common_topaz_v1:mixerdrv.obj
 0001:00002c60       ??_C@_1EM@KGOHBNDE@?$AAM?$AAI?$AAX?$AAE?$AAR?$AAC?$AAO?$AAN?$AAT?$AAR?$AAO?$AAL?$AA_?$AAC?$AAO?$AAN?$AAT?$AAR?$AAO?$AAL?$AAT?$AAY?$AAP?$AAE?$AA_?$AAS?$AAI?$AAN?$AAG?$AAL?$AAE?$AAS@ 10003c60     wavedev2_common_topaz_v1:mixerdrv.obj
 0001:00002cac       ??_C@_1DK@HHCAMDON@?$AAM?$AAI?$AAX?$AAE?$AAR?$AAC?$AAO?$AAN?$AAT?$AAR?$AAO?$AAL?$AA_?$AAC?$AAO?$AAN?$AAT?$AAR?$AAO?$AAL?$AAT?$AAY?$AAP?$AAE?$AA_?$AAM?$AAU?$AAX?$AA?$AA@ 10003cac     wavedev2_common_topaz_v1:mixerdrv.obj
 0001:00002ce8       ??_C@_1FA@ECHLHCDJ@?$AAM?$AAI?$AAX?$AAE?$AAR?$AAC?$AAO?$AAN?$AAT?$AAR?$AAO?$AAL?$AA_?$AAC?$AAO?$AAN?$AAT?$AAR?$AAO?$AAL?$AAT?$AAY?$AAP?$AAE?$AA_?$AAM?$AAU?$AAL?$AAT?$AAI?$AAP?$AAL@ 10003ce8     wavedev2_common_topaz_v1:mixerdrv.obj
 0001:00002d38       ??_C@_1DO@OPBKEMFB@?$AAM?$AAI?$AAX?$AAE?$AAR?$AAC?$AAO?$AAN?$AAT?$AAR?$AAO?$AAL?$AA_?$AAC?$AAO?$AAN?$AAT?$AAR?$AAO?$AAL?$AAT?$AAY?$AAP?$AAE?$AA_?$AAM?$AAI?$AAX?$AAE?$AAR?$AA?$AA@ 10003d38     wavedev2_common_topaz_v1:mixerdrv.obj
 0001:00002d78       ??_C@_1EA@BGMJCECN@?$AAM?$AAI?$AAX?$AAE?$AAR?$AAC?$AAO?$AAN?$AAT?$AAR?$AAO?$AAL?$AA_?$AAC?$AAO?$AAN?$AAT?$AAR?$AAO?$AAL?$AAT?$AAY?$AAP?$AAE?$AA_?$AAV?$AAO?$AAL?$AAU?$AAM?$AAE?$AA?$AA@ 10003d78     wavedev2_common_topaz_v1:mixerdrv.obj
 0001:00002db8       ??_C@_1EA@CECHMMMP@?$AAM?$AAI?$AAX?$AAE?$AAR?$AAC?$AAO?$AAN?$AAT?$AAR?$AAO?$AAL?$AA_?$AAC?$AAO?$AAN?$AAT?$AAR?$AAO?$AAL?$AAT?$AAY?$AAP?$AAE?$AA_?$AAT?$AAR?$AAE?$AAB?$AAL?$AAE?$AA?$AA@ 10003db8     wavedev2_common_topaz_v1:mixerdrv.obj
 0001:00002df8       ??_C@_1DO@KGELIMMP@?$AAM?$AAI?$AAX?$AAE?$AAR?$AAC?$AAO?$AAN?$AAT?$AAR?$AAO?$AAL?$AA_?$AAC?$AAO?$AAN?$AAT?$AAR?$AAO?$AAL?$AAT?$AAY?$AAP?$AAE?$AA_?$AAF?$AAA?$AAD?$AAE?$AAR?$AA?$AA@ 10003df8     wavedev2_common_topaz_v1:mixerdrv.obj
 0001:00002e38       ??_C@_1EG@NLNANFDC@?$AAM?$AAI?$AAX?$AAE?$AAR?$AAC?$AAO?$AAN?$AAT?$AAR?$AAO?$AAL?$AA_?$AAC?$AAO?$AAN?$AAT?$AAR?$AAO?$AAL?$AAT?$AAY?$AAP?$AAE?$AA_?$AAE?$AAQ?$AAU?$AAA?$AAL?$AAI?$AAZ@ 10003e38     wavedev2_common_topaz_v1:mixerdrv.obj
 0001:00002e80       ??_C@_1DM@FDDIFNFI@?$AAM?$AAI?$AAX?$AAE?$AAR?$AAC?$AAO?$AAN?$AAT?$AAR?$AAO?$AAL?$AA_?$AAC?$AAO?$AAN?$AAT?$AAR?$AAO?$AAL?$AAT?$AAY?$AAP?$AAE?$AA_?$AAB?$AAA?$AAS?$AAS?$AA?$AA@ 10003e80     wavedev2_common_topaz_v1:mixerdrv.obj
 0001:00002ec0       ??_C@_1EA@IAIECAKO@?$AAM?$AAI?$AAX?$AAE?$AAR?$AAC?$AAO?$AAN?$AAT?$AAR?$AAO?$AAL?$AA_?$AAC?$AAO?$AAN?$AAT?$AAR?$AAO?$AAL?$AAT?$AAY?$AAP?$AAE?$AA_?$AAC?$AAU?$AAS?$AAT?$AAO?$AAM?$AA?$AA@ 10003ec0     wavedev2_common_topaz_v1:mixerdrv.obj
 0001:00002fbc       ?m_cControls@MixerControlList@@0KB 10003fbc     wavedev2_common_topaz_v1:mixerdrv.obj
 0001:00002fc0       ??_C@_1BE@ELICABCK@?$AA?$DM?$AAu?$AAn?$AAk?$AAn?$AAo?$AAw?$AAn?$AA?$DO?$AA?$AA@ 10003fc0     wavedev2_common_topaz_v1:mixerdrv.obj
 0001:00002fd4       ??_C@_1CI@HHNFIEHC@?$AAM?$AAi?$AAx?$AAe?$AAr?$AAC?$AAa?$AAl?$AAl?$AAb?$AAa?$AAc?$AAk?$AA?$CI?$AA?$CF?$AAd?$AA?$CJ?$AA?$AN?$AA?6?$AA?$AA@ 10003fd4     wavedev2_common_topaz_v1:mixerdrv.obj
 0001:00002ffc       ??_C@_1BI@DKACBKCL@?$AAA?$AAu?$AAd?$AAi?$AAo?$AA?5?$AAM?$AAi?$AAx?$AAe?$AAr?$AA?$AA@ 10003ffc     wavedev2_common_topaz_v1:mixerdrv.obj
 0001:00003018       ??_C@_1FE@BDJOHFBK@?$AA?$FL?$AAE?$AAR?$AAR?$AAO?$AAR?$AA?$FN?$AA?5?$AA?$CC?$AAw?$AAd?$AAe?$AAv?$AA_?$AAM?$AAX?$AAD?$AAM?$AA_?$AAO?$AAP?$AAE?$AAN?$AA?3?$AA?5?$AAo?$AAu?$AAt?$AA?5?$AAo?$AAf?$AA?5@ 10004018     wavedev2_common_topaz_v1:mixerdrv.obj
 0001:0000306c       ??_C@_1DM@CHMELAAB@?$AAG?$AAe?$AAt?$AAM?$AAi?$AAx?$AAe?$AAr?$AAL?$AAi?$AAn?$AAe?$AAI?$AAn?$AAf?$AAo?$AA?3?$AA?5?$AA?$CC?$AA?$CF?$AAs?$AA?$CC?$AA?5?$AA?$CF?$AA0?$AA8?$AAx?$AA?$AN?$AA?6?$AA?$AA@ 1000406c     wavedev2_common_topaz_v1:mixerdrv.obj
 0001:000030a8       ??_C@_1FC@LHNBJHH@?$AAG?$AAe?$AAt?$AAM?$AAi?$AAx?$AAe?$AAr?$AAL?$AAi?$AAn?$AAe?$AAI?$AAn?$AAf?$AAo?$AA?3?$AA?5?$AAi?$AAn?$AAv?$AAa?$AAl?$AAi?$AAd?$AA?5?$AAl?$AAi?$AAn?$AAe?$AA?5?$AAI@ 100040a8     wavedev2_common_topaz_v1:mixerdrv.obj
 0001:00003100       ??_C@_1GA@DDKINBEJ@?$AAG?$AAe?$AAt?$AAM?$AAi?$AAx?$AAe?$AAr?$AAL?$AAi?$AAn?$AAe?$AAI?$AAn?$AAf?$AAo?$AA?3?$AA?5?$AAn?$AAo?$AA?5?$AAl?$AAi?$AAn?$AAe?$AA?5?$AAo?$AAf?$AA?5?$AAt?$AAa?$AAr@ 10004100     wavedev2_common_topaz_v1:mixerdrv.obj
 0001:00003160       ??_C@_1GG@MELCAJPL@?$AAG?$AAe?$AAt?$AAM?$AAi?$AAx?$AAe?$AAr?$AAL?$AAi?$AAn?$AAe?$AAI?$AAn?$AAf?$AAo?$AA?3?$AA?5?$AAn?$AAo?$AA?5?$AAl?$AAi?$AAn?$AAe?$AA?5?$AAo?$AAf?$AA?5?$AAc?$AAo?$AAm@ 10004160     wavedev2_common_topaz_v1:mixerdrv.obj
 0001:000031c8       ??_C@_1EO@HDKNAFNG@?$AAG?$AAe?$AAt?$AAM?$AAi?$AAx?$AAe?$AAr?$AAL?$AAi?$AAn?$AAe?$AAI?$AAn?$AAf?$AAo?$AA?3?$AA?5?$AAi?$AAn?$AAv?$AAa?$AAl?$AAi?$AAd?$AA?5?$AAq?$AAu?$AAe?$AAr?$AAy?$AA?5@ 100041c8     wavedev2_common_topaz_v1:mixerdrv.obj
 0001:00003218       ??_C@_1DE@PIKBGEIJ@?$AAG?$AAe?$AAt?$AAM?$AAi?$AAx?$AAe?$AAr?$AAL?$AAi?$AAn?$AAe?$AAI?$AAn?$AAf?$AAo?$AA?5?$AAT?$AAA?$AAR?$AAG?$AAE?$AAT?$AA?$AN?$AA?6?$AA?$AA@ 10004218     wavedev2_common_topaz_v1:mixerdrv.obj
 0001:0000324c       ??_C@_1DK@COFPEFKO@?$AAG?$AAe?$AAt?$AAM?$AAi?$AAx?$AAe?$AAr?$AAL?$AAi?$AAn?$AAe?$AAI?$AAn?$AAf?$AAo?$AA?5?$AAC?$AAO?$AAM?$AAP?$AAO?$AAN?$AAE?$AAN?$AAT?$AA?$AN?$AA?6?$AA?$AA@ 1000424c     wavedev2_common_topaz_v1:mixerdrv.obj
 0001:00003288       ??_C@_1FG@LCCLAGKB@?$AAG?$AAe?$AAt?$AAM?$AAi?$AAx?$AAe?$AAr?$AAL?$AAi?$AAn?$AAe?$AAI?$AAn?$AAf?$AAo?$AA?3?$AA?5?$AAi?$AAn?$AAv?$AAa?$AAl?$AAi?$AAd?$AA?5?$AAs?$AAo?$AAu?$AAr?$AAc?$AAe@ 10004288     wavedev2_common_topaz_v1:mixerdrv.obj
 0001:000032e0       ??_C@_1HG@JHFCMAJM@?$AAG?$AAe?$AAt?$AAM?$AAi?$AAx?$AAe?$AAr?$AAL?$AAi?$AAn?$AAe?$AAI?$AAn?$AAf?$AAo?$AA?3?$AA?5?$AAi?$AAn?$AAc?$AAo?$AAn?$AAs?$AAi?$AAs?$AAt?$AAe?$AAn?$AAt?$AA?5?$AAi@ 100042e0     wavedev2_common_topaz_v1:mixerdrv.obj
 0001:00003358       ??_C@_1EA@IAOAGGKE@?$AAG?$AAe?$AAt?$AAM?$AAi?$AAx?$AAe?$AAr?$AAL?$AAi?$AAn?$AAe?$AAI?$AAn?$AAf?$AAo?$AA?5?$AAS?$AAO?$AAU?$AAR?$AAC?$AAE?$AA?5?$AA?$CF?$AAx?$AA?5?$AA?$CF?$AAx?$AA?$AN?$AA?6?$AA?$AA@ 10004358     wavedev2_common_topaz_v1:mixerdrv.obj
 0001:00003398       ??_C@_1DK@GMMCEECL@?$AAG?$AAe?$AAt?$AAM?$AAi?$AAx?$AAe?$AAr?$AAL?$AAi?$AAn?$AAe?$AAI?$AAn?$AAf?$AAo?$AA?5?$AAL?$AAI?$AAN?$AAE?$AAI?$AAD?$AA?5?$AA?$CF?$AAx?$AA?$AN?$AA?6?$AA?$AA@ 10004398     wavedev2_common_topaz_v1:mixerdrv.obj
 0001:000033d8       ??_C@_1GA@BBJIEEAD@?$AAG?$AAe?$AAt?$AAM?$AAi?$AAx?$AAe?$AAr?$AAL?$AAi?$AAn?$AAe?$AAI?$AAn?$AAf?$AAo?$AA?3?$AA?5?$AAi?$AAn?$AAv?$AAa?$AAl?$AAi?$AAd?$AA?5?$AAd?$AAe?$AAs?$AAt?$AAi?$AAn@ 100043d8     wavedev2_common_topaz_v1:mixerdrv.obj
 0001:00003438       ??_C@_1EE@DGPNNKNM@?$AAG?$AAe?$AAt?$AAM?$AAi?$AAx?$AAe?$AAr?$AAL?$AAi?$AAn?$AAe?$AAI?$AAn?$AAf?$AAo?$AA?5?$AAD?$AAE?$AAS?$AAT?$AAI?$AAN?$AAA?$AAT?$AAI?$AAO?$AAN?$AA?5?$AA?$CF?$AAx?$AA?$AN@ 10004438     wavedev2_common_topaz_v1:mixerdrv.obj
 0001:00003480       ??_C@_1FG@OKMEMBEL@?$AAG?$AAe?$AAt?$AAM?$AAi?$AAx?$AAe?$AAr?$AAL?$AAi?$AAn?$AAe?$AAC?$AAo?$AAn?$AAt?$AAr?$AAo?$AAl?$AAs?$AA?3?$AA?5?$AAi?$AAn?$AAv?$AAa?$AAl?$AAi?$AAd?$AA?5?$AAq?$AAu@ 10004480     wavedev2_common_topaz_v1:mixerdrv.obj
 0001:000034d8       ??_C@_1IG@OCFKLJPN@?$AAG?$AAe?$AAt?$AAM?$AAi?$AAx?$AAe?$AAr?$AAL?$AAi?$AAn?$AAe?$AAC?$AAo?$AAn?$AAt?$AAr?$AAo?$AAl?$AAs?$AA?3?$AA?5?$AAl?$AAi?$AAn?$AAe?$AA?5?$AA?$CF?$AA0?$AA4?$AAx?$AA?5@ 100044d8     wavedev2_common_topaz_v1:mixerdrv.obj
 0001:00003560       ??_C@_1GO@CMCLLJCP@?$AAG?$AAe?$AAt?$AAM?$AAi?$AAx?$AAe?$AAr?$AAL?$AAi?$AAn?$AAe?$AAC?$AAo?$AAn?$AAt?$AAr?$AAo?$AAl?$AAs?$AA?3?$AA?5?$AAc?$AAo?$AAn?$AAt?$AAr?$AAo?$AAl?$AA?5?$AAc?$AAo@ 10004560     wavedev2_common_topaz_v1:mixerdrv.obj
 0001:000035d0       ??_C@_1EM@NAGBJFBM@?$AAG?$AAe?$AAt?$AAM?$AAi?$AAx?$AAe?$AAr?$AAL?$AAi?$AAn?$AAe?$AAC?$AAo?$AAn?$AAt?$AAr?$AAo?$AAl?$AAs?$AA?3?$AA?5?$AAO?$AAN?$AAE?$AAB?$AAY?$AAT?$AAY?$AAP?$AAE?$AA?5@ 100045d0     wavedev2_common_topaz_v1:mixerdrv.obj
 0001:00003620       ??_C@_1GM@MONMFDNB@?$AAG?$AAe?$AAt?$AAM?$AAi?$AAx?$AAe?$AAr?$AAL?$AAi?$AAn?$AAe?$AAC?$AAo?$AAn?$AAt?$AAr?$AAo?$AAl?$AAs?$AA?3?$AA?5?$AAc?$AAo?$AAn?$AAt?$AAr?$AAo?$AAl?$AA?5?$AAc?$AAo@ 10004620     wavedev2_common_topaz_v1:mixerdrv.obj
 0001:00003690       ??_C@_1EG@IPGPLBHF@?$AAG?$AAe?$AAt?$AAM?$AAi?$AAx?$AAe?$AAr?$AAL?$AAi?$AAn?$AAe?$AAC?$AAo?$AAn?$AAt?$AAr?$AAo?$AAl?$AAs?$AA?3?$AA?5?$AAO?$AAN?$AAE?$AAB?$AAY?$AAI?$AAD?$AA?5?$AA?$CF?$AAx@ 10004690     wavedev2_common_topaz_v1:mixerdrv.obj
 0001:000036d8       ??_C@_1JG@CANNPDPK@?$AAG?$AAe?$AAt?$AAM?$AAi?$AAx?$AAe?$AAr?$AAL?$AAi?$AAn?$AAe?$AAC?$AAo?$AAn?$AAt?$AAr?$AAo?$AAl?$AAs?$AA?3?$AA?5?$AAi?$AAn?$AAc?$AAo?$AAr?$AAr?$AAe?$AAc?$AAt?$AA?5@ 100046d8     wavedev2_common_topaz_v1:mixerdrv.obj
 0001:00003770       ??_C@_1FK@PFCBAFBC@?$AAG?$AAe?$AAt?$AAM?$AAi?$AAx?$AAe?$AAr?$AAL?$AAi?$AAn?$AAe?$AAC?$AAo?$AAn?$AAt?$AAr?$AAo?$AAl?$AAs?$AA?3?$AA?5?$AAi?$AAn?$AAv?$AAa?$AAl?$AAi?$AAd?$AA?5?$AAl?$AAi@ 10004770     wavedev2_common_topaz_v1:mixerdrv.obj
 0001:000037cc       ??_C@_1DO@KJNHEOOA@?$AAG?$AAe?$AAt?$AAM?$AAi?$AAx?$AAe?$AAr?$AAL?$AAi?$AAn?$AAe?$AAC?$AAo?$AAn?$AAt?$AAr?$AAo?$AAl?$AAs?$AA?3?$AA?5?$AAA?$AAL?$AAL?$AA?5?$AA?$CF?$AAx?$AA?$AN?$AA?6?$AA?$AA@ 100047cc     wavedev2_common_topaz_v1:mixerdrv.obj
 0001:0000380c       ??_C@_1DK@HNFPDNP@?$AAG?$AAe?$AAt?$AAM?$AAi?$AAx?$AAe?$AAr?$AAC?$AAo?$AAn?$AAt?$AAr?$AAo?$AAl?$AAD?$AAe?$AAt?$AAa?$AAi?$AAl?$AAs?$AA?$CI?$AA?$CF?$AAd?$AA?$CJ?$AA?$AN?$AA?6?$AA?$AA@ 1000480c     wavedev2_common_topaz_v1:mixerdrv.obj
 0001:00003848       ??_C@_1DK@IAOOCHGE@?$AAS?$AAe?$AAt?$AAM?$AAi?$AAx?$AAe?$AAr?$AAC?$AAo?$AAn?$AAt?$AAr?$AAo?$AAl?$AAD?$AAe?$AAt?$AAa?$AAi?$AAl?$AAs?$AA?$CI?$AA?$CF?$AAd?$AA?$CJ?$AA?$AN?$AA?6?$AA?$AA@ 10004848     wavedev2_common_topaz_v1:mixerdrv.obj
 0001:00003884       ??_7MixerControlList@@6B@  10004884     wavedev2_common_topaz_v1:mixerdrv.obj
 0001:00003888       ??_7MixerControlVolumeMaster@@6B@ 10004888     wavedev2_common_topaz_v1:mixerdrv.obj
 0001:000038ac       ??_7MixerControlVolume@@6B@ 100048ac     wavedev2_common_topaz_v1:mixerdrv.obj
 0001:000038d0       ??_7MixerControl@@6B@      100048d0     wavedev2_common_topaz_v1:mixerdrv.obj
 0001:000038f0       ??_C@_1GA@LNIMIIDM@?$AAS?$AAe?$AAt?$AAM?$AAi?$AAx?$AAe?$AAr?$AAC?$AAo?$AAn?$AAt?$AAr?$AAo?$AAl?$AAD?$AAe?$AAt?$AAa?$AAi?$AAl?$AAs?$AA?3?$AA?5?$AAV?$AAo?$AAl?$AAu?$AAm?$AAe?$AA?5?$AAe@ 100048f0     wavedev2_common_topaz_v1:mixerdrv.obj
 0001:00003950       ??_C@_1BM@DBCMFCBE@?$AAM?$AAa?$AAs?$AAt?$AAe?$AAr?$AA?5?$AAV?$AAo?$AAl?$AAu?$AAm?$AAe?$AA?$AA@ 10004950     wavedev2_common_topaz_v1:mixerdrv.obj
 0001:0000396c       ??_7MixerControlVolumeMic@@6B@ 1000496c     wavedev2_common_topaz_v1:mixerdrv.obj
 0001:00003990       ??_C@_1BG@LAGONMFD@?$AAM?$AAi?$AAc?$AA?5?$AAV?$AAo?$AAl?$AAu?$AAm?$AAe?$AA?$AA@ 10004990     wavedev2_common_topaz_v1:mixerdrv.obj
 0001:000039a8       ??_7MixerControlMuteMaster@@6B@ 100049a8     wavedev2_common_topaz_v1:mixerdrv.obj
 0001:000039cc       ??_7MixerControlBoolean@@6B@ 100049cc     wavedev2_common_topaz_v1:mixerdrv.obj
 0001:000039f0       ??_C@_1BI@PEAJCPFH@?$AAM?$AAa?$AAs?$AAt?$AAe?$AAr?$AA?5?$AAM?$AAu?$AAt?$AAe?$AA?$AA@ 100049f0     wavedev2_common_topaz_v1:mixerdrv.obj
 0001:00003a08       ??_7MixerControlMuteMic@@6B@ 10004a08     wavedev2_common_topaz_v1:mixerdrv.obj
 0001:00003a2c       ??_C@_1BC@MOMKCGGI@?$AAM?$AAi?$AAc?$AA?5?$AAM?$AAu?$AAt?$AAe?$AA?$AA@ 10004a2c     wavedev2_common_topaz_v1:mixerdrv.obj
 0001:00003a40       ??_7MixerControlLoopback@@6B@ 10004a40     wavedev2_common_topaz_v1:mixerdrv.obj
 0001:00003a64       ??_C@_1BC@NMCMBANA@?$AAL?$AAo?$AAo?$AAp?$AAb?$AAa?$AAc?$AAk?$AA?$AA@ 10004a64     wavedev2_common_topaz_v1:mixerdrv.obj
 0001:00003a78       ??_C@_1CC@NMFCMAHN@?$AAL?$AAo?$AAo?$AAp?$AAb?$AAa?$AAc?$AAk?$AA?5?$AAC?$AAo?$AAn?$AAt?$AAr?$AAo?$AAl?$AA?$AA@ 10004a78     wavedev2_common_topaz_v1:mixerdrv.obj
 0001:00003a9c       ??_7MixerControlInputMux@@6B@ 10004a9c     wavedev2_common_topaz_v1:mixerdrv.obj
 0001:00003ab8       ??_C@_1BE@FNMPOHBO@?$AAI?$AAn?$AAp?$AAu?$AAt?$AA?5?$AAM?$AAu?$AAx?$AA?$AA@ 10004ab8     wavedev2_common_topaz_v1:mixerdrv.obj
 0001:00003ad0       ??_C@_1EM@DBPFHEAH@?$AA?$FL?$AAE?$AAR?$AAR?$AAO?$AAR?$AA?$FN?$AA?5?$AA?$CC?$AAU?$AAn?$AAs?$AAu?$AAp?$AAp?$AAo?$AAr?$AAt?$AAe?$AAd?$AA?5?$AAm?$AAi?$AAx?$AAe?$AAr?$AA?5?$AAm?$AAe?$AAs?$AAs?$AAa@ 10004ad0     wavedev2_common_topaz_v1:mixerdrv.obj
 0001:00003b1c       ??_C@_1DC@MEFIDC@?$AAM?$AAX?$AAD?$AAM?$AA_?$AAS?$AAE?$AAT?$AAC?$AAO?$AAN?$AAT?$AAR?$AAO?$AAL?$AAD?$AAE?$AAT?$AAA?$AAI?$AAL?$AAS?$AA?$AN?$AA?6?$AA?$AA@ 10004b1c     wavedev2_common_topaz_v1:mixerdrv.obj
 0001:00003b50       ??_C@_1DC@CEKCBIBD@?$AAM?$AAX?$AAD?$AAM?$AA_?$AAG?$AAE?$AAT?$AAC?$AAO?$AAN?$AAT?$AAR?$AAO?$AAL?$AAD?$AAE?$AAT?$AAA?$AAI?$AAL?$AAS?$AA?$AN?$AA?6?$AA?$AA@ 10004b50     wavedev2_common_topaz_v1:mixerdrv.obj
 0001:00003b84       ??_C@_1CO@OJFEDBFL@?$AAM?$AAX?$AAD?$AAM?$AA_?$AAG?$AAE?$AAT?$AAL?$AAI?$AAN?$AAE?$AAC?$AAO?$AAN?$AAT?$AAR?$AAO?$AAL?$AAS?$AA?$AN?$AA?6?$AA?$AA@ 10004b84     wavedev2_common_topaz_v1:mixerdrv.obj
 0001:00003bb4       ??_C@_1CG@CLPEJCBP@?$AAM?$AAX?$AAD?$AAM?$AA_?$AAG?$AAE?$AAT?$AAL?$AAI?$AAN?$AAE?$AAI?$AAN?$AAF?$AAO?$AA?$AN?$AA?6?$AA?$AA@ 10004bb4     wavedev2_common_topaz_v1:mixerdrv.obj
 0001:00003bdc       ??_C@_1BK@DOLEBCGM@?$AAM?$AAX?$AAD?$AAM?$AA_?$AAC?$AAL?$AAO?$AAS?$AAE?$AA?$AN?$AA?6?$AA?$AA@ 10004bdc     wavedev2_common_topaz_v1:mixerdrv.obj
 0001:00003bf8       ??_C@_1BI@FCEHOKDK@?$AAM?$AAX?$AAD?$AAM?$AA_?$AAO?$AAP?$AAE?$AAN?$AA?$AN?$AA?6?$AA?$AA@ 10004bf8     wavedev2_common_topaz_v1:mixerdrv.obj
 0001:00003c10       ??_C@_1CE@NFMKBKIL@?$AAM?$AAX?$AAD?$AAM?$AA_?$AAG?$AAE?$AAT?$AAD?$AAE?$AAV?$AAC?$AAA?$AAP?$AAS?$AA?$AN?$AA?6?$AA?$AA@ 10004c10     wavedev2_common_topaz_v1:mixerdrv.obj
 0001:00003c34       ??_C@_1CE@HLFFBCHG@?$AAM?$AAX?$AAD?$AAM?$AA_?$AAG?$AAE?$AAT?$AAN?$AAU?$AAM?$AAD?$AAE?$AAV?$AAS?$AA?$AN?$AA?6?$AA?$AA@ 10004c34     wavedev2_common_topaz_v1:mixerdrv.obj
 0001:00003c58       ?ms_BasePitchTable@CMidiStream@@0QBKB 10004c58     wavedev2_common_topaz_v1:midistrm.obj
 0001:00003c88       ??_C@_1HC@PLGDHHAP@?$AAE?$AAX?$AAC?$AAE?$AAP?$AAT?$AAI?$AAO?$AAN?$AA?5?$AAI?$AAN?$AA?5?$AAI?$AAS?$AAT?$AA?5?$AAf?$AAo?$AAr?$AA?5?$AAm?$AAi?$AAd?$AAi?$AA?5?$AAs?$AAt?$AAr?$AAe?$AAa?$AAm@ 10004c88     wavedev2_common_topaz_v1:midistrm.obj
 0001:00003d00       ?SineTable@CMidiNote@@0QBFB 10004d00     wavedev2_common_topaz_v1:midinote.obj
 0001:00003f08       ??_C@_1JM@CHBKJEIO@?$AAC?$AAM?$AAi?$AAd?$AAi?$AAN?$AAo?$AAt?$AAe?$AA?3?$AA?3?$AAN?$AAo?$AAt?$AAe?$AAO?$AAf?$AAf?$AA?0?$AA?5?$AAm?$AA_?$AAI?$AAn?$AAd?$AAe?$AAx?$AA?5?$AA?$DN?$AA?5?$AA0?$AAx@ 10004f08     wavedev2_common_topaz_v1:midinote.obj
 0001:00003fa8       ??_C@_1GO@GPNNNFCM@?$AAC?$AAM?$AAi?$AAd?$AAi?$AAN?$AAo?$AAt?$AAe?$AA?3?$AA?3?$AAR?$AAe?$AAn?$AAd?$AAe?$AAr?$AA?0?$AA?5?$AAL?$AAa?$AAs?$AAt?$AA?5?$AAi?$AAn?$AAd?$AAe?$AAx?$AA?5?$AAa?$AAf@ 10004fa8     wavedev2_common_topaz_v1:midinote.obj
 0001:00004018       ??_C@_1HC@ICNNALDK@?$AAC?$AAM?$AAi?$AAd?$AAi?$AAN?$AAo?$AAt?$AAe?$AA?3?$AA?3?$AAR?$AAe?$AAn?$AAd?$AAe?$AAr?$AA?0?$AA?5?$AAN?$AAo?$AAt?$AAe?$AA?5?$AAi?$AAn?$AA?5?$AAr?$AAe?$AAl?$AAe?$AAa@ 10005018     wavedev2_common_topaz_v1:midinote.obj
 0001:000040bc       ?BSPAudioStartDAC@@YAXXZ   100050bc f   bsphwctxt.obj
 0001:000040dc       ?BSPAudioStopDAC@@YAXXZ    100050dc f   bsphwctxt.obj
 0001:000040fc       ?BSPAudioStartADC@@YAXXZ   100050fc f   bsphwctxt.obj
 0001:0000411c       ?BSPAudioStopADC@@YAXXZ    1000511c f   bsphwctxt.obj
 0001:0000413c       ?BSPSetSpeakerEnable@@YAXH@Z 1000513c f   bsphwctxt.obj
 0001:00004190       ?BSPAudioSelectADCSource@@YAXK@Z 10005190 f   bsphwctxt.obj
 0001:000041d8       ?BSPAudioSetCodecLoopback@@YAHH@Z 100051d8 f   bsphwctxt.obj
 0001:00004200       ?BSPAudioSetOutputGain@@YAXK@Z 10005200 f   bsphwctxt.obj
 0001:000043e8       ?BSPAudioSetInputGain@@YAXK@Z 100053e8 f   bsphwctxt.obj
 0001:00004468       ?BSPAudioGetInputDeviceNum@@YAEXZ 10005468 f   bsphwctxt.obj
 0001:00004480       ?BSPAllocOutputDMABuffer@@YAGPAPAEPAT_LARGE_INTEGER@@@Z 10005480 f   bsphwctxt.obj
 0001:000044f8       ?BSPDeallocOutputDMABuffer@@YAXPAE@Z 100054f8 f   bsphwctxt.obj
 0001:0000450c       ?BSPAllocInputDMABuffer@@YAGPAPAEPAT_LARGE_INTEGER@@@Z 1000550c f   bsphwctxt.obj
 0001:00004578       ?BSPDeallocInputDMABuffer@@YAXPAE@Z 10005578 f   bsphwctxt.obj
 0001:000045e8       ?BSPAudioIomuxConfig@@YAXXZ 100055e8 f   bsphwctxt.obj
 0001:00004634       ?BSPSsiEnableClock@@YAHIH@Z 10005634 f   bsphwctxt.obj
 0001:000046e0       ?BSPAudmuxEnableClock@@YAHH@Z 100056e0 f   bsphwctxt.obj
 0001:00004744       ?BSPGetAudmuxIntPort@@YA?AW4AUDMUX_INTERNAL_PORT@@XZ 10005744 f   bsphwctxt.obj
 0001:0000475c       ?BSPGetAudmuxExtPort@@YA?AW4AUDMUX_EXTERNAL_PORT@@XZ 1000575c f   bsphwctxt.obj
 0001:00004774       ?BSPAudioGetSdmaPriority@@YAEXZ 10005774 f   bsphwctxt.obj
 0001:0000478c       ?BSPAudioPowerUp@@YAXH@Z   1000578c f   bsphwctxt.obj
 0001:000047c0       ?BSPAudioPowerDown@@YAXH@Z 100057c0 f   bsphwctxt.obj
 0001:000047f4       ?BSPAudioGetProtocol@@YA?AW4AUDIO_PROTOCOL@@XZ 100057f4 f   bsphwctxt.obj
 0001:0000480c       ?BSPAudioDeinitCodec@@YAXXZ 1000580c f   bsphwctxt.obj
 0001:00004888       ?BSPAudioInitCodec@@YAHXZ  10005888 f   bsphwctxt.obj
 0001:0000496c       ?BSPIsHeadphoneDetectSupported@@YAHXZ 1000596c f   bsphwctxt.obj
 0001:00004984       ?BSPGetHPDetectIRQ@@YAKXZ  10005984 f   bsphwctxt.obj
 0001:0000499c       ?BSPAudioHandleHPDetectIRQ@@YAXXZ 1000599c f   bsphwctxt.obj
 0001:000049a0       ?BSPGetBitsPerSample@@YAGXZ 100059a0 f   bsphwctxt.obj
 0001:000049c0       ??_GSGTL5000Codec@@QAAPAXI@Z 100059c0 f i bsphwctxt.obj
 0001:00004a04       ??0SGTL5000Codec@@QAA@XZ   10005a04 f   sgtl5000codec.obj
 0001:00004a84       ??1SGTL5000Codec@@QAA@XZ   10005a84 f   sgtl5000codec.obj
 0001:00004ab4       ?SGTL5000I2CInit@SGTL5000Codec@@QAAIXZ 10005ab4 f   sgtl5000codec.obj
 0001:00004be0       ?SGTL5000I2CClose@SGTL5000Codec@@QAAXXZ 10005be0 f   sgtl5000codec.obj
 0001:00004c38       ?SGTL5000WriteRegister@SGTL5000Codec@@QAAIGG@Z 10005c38 f   sgtl5000codec.obj
 0001:00004d64       ?SGTL5000ReadRegister@SGTL5000Codec@@QAAIGPAG@Z 10005d64 f   sgtl5000codec.obj
 0001:00004eb8       ?SGTL5000ModifyRegister@SGTL5000Codec@@QAAIGGG@Z 10005eb8 f   sgtl5000codec.obj
 0001:00004f78       ?SGTL5000CodecInit@SGTL5000Codec@@QAAIXZ 10005f78 f   sgtl5000codec.obj
 0001:00005298       ?SGTL5000ConfigureDuplexMode@SGTL5000Codec@@QAAXXZ 10006298 f   sgtl5000codec.obj
 0001:0000532c       ?SGTL5000ConfigureLoopbackMode@SGTL5000Codec@@QAAXXZ 1000632c f   sgtl5000codec.obj
 0001:00005400       ?SGTL5000ConfigurePowerMode@SGTL5000Codec@@QAAXG@Z 10006400 f   sgtl5000codec.obj
 0001:000058cc       ?SGTL5000RampHPVolume@SGTL5000Codec@@QAAXG@Z 100068cc f   sgtl5000codec.obj
 0001:00005a28       ?SGTL5000SetDACPower@SGTL5000Codec@@QAAXG@Z 10006a28 f   sgtl5000codec.obj
 0001:00005a84       ?SGTL5000SetADCPower@SGTL5000Codec@@QAAXG@Z 10006a84 f   sgtl5000codec.obj
 0001:00005aec       ?SGTL5000SetLINEOUTPower@SGTL5000Codec@@QAAXG@Z 10006aec f   sgtl5000codec.obj
 0001:00005b3c       ?SGTL5000SetHPOUTPower@SGTL5000Codec@@QAAXGG@Z 10006b3c f   sgtl5000codec.obj
 0001:00005ba4       ?SGTL5000SetSampleRate@SGTL5000Codec@@QAAXW4SGTL5000_SAMPLE_RATE@@@Z 10006ba4 f   sgtl5000codec.obj
 0001:00005c00       ?SGTL5000SetDACVolume@SGTL5000Codec@@QAAXEE@Z 10006c00 f   sgtl5000codec.obj
 0001:00005c50       ?SGTL5000SetADCVolume@SGTL5000Codec@@QAAXEE@Z 10006c50 f   sgtl5000codec.obj
 0001:00005cb4       ?SGTL5000DACMute@SGTL5000Codec@@QAAXG@Z 10006cb4 f   sgtl5000codec.obj
 0001:00005d20       ?SGTL5000HPMute@SGTL5000Codec@@QAAXG@Z 10006d20 f   sgtl5000codec.obj
 0001:00005d7c       ?SGTL5000LineOutMute@SGTL5000Codec@@QAAXG@Z 10006d7c f   sgtl5000codec.obj
 0001:00005dd8       ?SGTL5000ADCMute@SGTL5000Codec@@QAAXG@Z 10006dd8 f   sgtl5000codec.obj
 0001:00005e28       ?SGTL5000SetADCInput@SGTL5000Codec@@QAAXW4SGTL5000_ADC_INPUT@@@Z 10006e28 f   sgtl5000codec.obj
 0001:00005e94       ?SGTL5000HPDetected@SGTL5000Codec@@QAAXI@Z 10006e94 f   sgtl5000codec.obj
 0001:00005eb8       ?SGTL5000ForceSpeaker@SGTL5000Codec@@QAAXI@Z 10006eb8 f   sgtl5000codec.obj
 0001:00005edc       ?SGTL5000SpeakerHeadphoneSelection@SGTL5000Codec@@QAAXXZ 10006edc f   sgtl5000codec.obj
 0001:00005f4c       ?SGTL5000DumpRegisters@SGTL5000Codec@@QAAXXZ 10006f4c f   sgtl5000codec.obj
 0001:00006a60       DllMain                    10007a60 f   wavedev2_common_topaz_v1:wavemain.obj
 0001:00006ab0       WAV_Init                   10007ab0 f   wavedev2_common_topaz_v1:wavemain.obj
 0001:00006ae4       WAV_Deinit                 10007ae4 f   wavedev2_common_topaz_v1:wavemain.obj
 0001:00006b20       WAV_Open                   10007b20 f   wavedev2_common_topaz_v1:wavemain.obj
 0001:00006b88       WAV_Close                  10007b88 f   wavedev2_common_topaz_v1:wavemain.obj
 0001:00006bc8       ?HandleWaveMessage@@YAHPAUMMDRV_MESSAGE_PARAMS@@PAK@Z 10007bc8 f   wavedev2_common_topaz_v1:wavemain.obj
 0001:00007570       WAV_IOControl              10008570 f   wavedev2_common_topaz_v1:wavemain.obj
 0001:00007728       ?Lock@HardwareContext@@QAAXXZ 10008728 f i wavedev2_common_topaz_v1:wavemain.obj
 0001:00007748       ?Unlock@HardwareContext@@QAAXXZ 10008748 f i wavedev2_common_topaz_v1:wavemain.obj
 0001:00007768       ?GetNumInputDevices@HardwareContext@@QAAKXZ 10008768 f i wavedev2_common_topaz_v1:wavemain.obj
 0001:00007798       ?GetNumOutputDevices@HardwareContext@@QAAKXZ 10008798 f i wavedev2_common_topaz_v1:wavemain.obj
 0001:000077c0       ?GetInputDeviceContext@HardwareContext@@QAAPAVDeviceContext@@I@Z 100087c0 f i wavedev2_common_topaz_v1:wavemain.obj
 0001:000077ec       ?GetOutputDeviceContext@HardwareContext@@QAAPAVDeviceContext@@I@Z 100087ec f i wavedev2_common_topaz_v1:wavemain.obj
 0001:00007818       ?CreateHWContext@HardwareContext@@SAHK@Z 10008818 f   wavedev2_common_topaz_v1:hwctxt.obj
 0001:000078dc       ??0HardwareContext@@QAA@XZ 100088dc f   wavedev2_common_topaz_v1:hwctxt.obj
 0001:00007970       ??1HardwareContext@@QAA@XZ 10008970 f   wavedev2_common_topaz_v1:hwctxt.obj
 0001:00007990       ?Init@HardwareContext@@QAAHK@Z 10008990 f   wavedev2_common_topaz_v1:hwctxt.obj
 0001:00007eac       ?Deinit@HardwareContext@@QAAHXZ 10008eac f   wavedev2_common_topaz_v1:hwctxt.obj
 0001:00008068       ?InitSsi@HardwareContext@@AAAXW4AUDIO_PROTOCOL@@@Z 10009068 f   wavedev2_common_topaz_v1:hwctxt.obj
 0001:00008300       ?InitAudmux@HardwareContext@@AAAXW4AUDMUX_INTERNAL_PORT@@W4AUDMUX_EXTERNAL_PORT@@@Z 10009300 f   wavedev2_common_topaz_v1:hwctxt.obj
 0001:0000842c       ?InitOutputDMA@HardwareContext@@AAAHXZ 1000942c f   wavedev2_common_topaz_v1:hwctxt.obj
 0001:0000886c       ?InitInputDMA@HardwareContext@@AAAHXZ 1000986c f   wavedev2_common_topaz_v1:hwctxt.obj
 0001:00008cfc       ?InitInterruptThread@HardwareContext@@IAAHXZ 10009cfc f   wavedev2_common_topaz_v1:hwctxt.obj
 0001:00008e28       ?InitHPDetectInterruptThread@HardwareContext@@IAAHXZ 10009e28 f   wavedev2_common_topaz_v1:hwctxt.obj
 0001:00008fc0       ?InitDisableDelayThread@HardwareContext@@IAAHXZ 10009fc0 f   wavedev2_common_topaz_v1:hwctxt.obj
 0001:00009208       ?StartCodec@HardwareContext@@AAAXW4AUDIO_BUS@@@Z 1000a208 f   wavedev2_common_topaz_v1:hwctxt.obj
 0001:00009234       ?StopCodec@HardwareContext@@AAAXW4AUDIO_BUS@@@Z 1000a234 f   wavedev2_common_topaz_v1:hwctxt.obj
 0001:00009368       ?StartSsi@HardwareContext@@AAAXW4AUDIO_BUS@@@Z 1000a368 f   wavedev2_common_topaz_v1:hwctxt.obj
 0001:000095ec       ?StopSsi@HardwareContext@@AAAXW4AUDIO_BUS@@@Z 1000a5ec f   wavedev2_common_topaz_v1:hwctxt.obj
 0001:00009894       ?StartOutputDMA@HardwareContext@@QAAHXZ 1000a894 f   wavedev2_common_topaz_v1:hwctxt.obj
 0001:00009b28       ?StopOutputDMA@HardwareContext@@QAAXXZ 1000ab28 f   wavedev2_common_topaz_v1:hwctxt.obj
 0001:00009bbc       ?StartInputDMA@HardwareContext@@QAAHXZ 1000abbc f   wavedev2_common_topaz_v1:hwctxt.obj
 0001:00009dec       ?StopInputDMA@HardwareContext@@QAAXXZ 1000adec f   wavedev2_common_topaz_v1:hwctxt.obj
 0001:00009e84       ?TransferOutputBuffers@HardwareContext@@IAAKXZ 1000ae84 f   wavedev2_common_topaz_v1:hwctxt.obj
 0001:00009f7c       ?TransferInputBuffers@HardwareContext@@IAAKE@Z 1000af7c f   wavedev2_common_topaz_v1:hwctxt.obj
 0001:0000a10c       ?TransferBuffer@HardwareContext@@IAAKW4AUDIO_BUS@@E@Z 1000b10c f   wavedev2_common_topaz_v1:hwctxt.obj
 0001:0000a268       ?InterruptThread@HardwareContext@@QAAXXZ 1000b268 f   wavedev2_common_topaz_v1:hwctxt.obj
 0001:0000a33c       ?HPDetectInterruptThread@HardwareContext@@QAAXXZ 1000b33c f   wavedev2_common_topaz_v1:hwctxt.obj
 0001:0000a3ec       ?OutputIntrRoutine@HardwareContext@@AAAXXZ 1000b3ec f   wavedev2_common_topaz_v1:hwctxt.obj
 0001:0000a6c8       ?InputIntrRoutine@HardwareContext@@AAAXXZ 1000b6c8 f   wavedev2_common_topaz_v1:hwctxt.obj
 0001:0000aa38       ?DisableDelayThread@HardwareContext@@QAAXXZ 1000ba38 f   wavedev2_common_topaz_v1:hwctxt.obj
 0001:0000aca0       ?CallInterruptThread@@YAXPAVHardwareContext@@@Z 1000bca0 f   wavedev2_common_topaz_v1:hwctxt.obj
 0001:0000acbc       ?CallDisableDelayThread@@YAXPAVHardwareContext@@@Z 1000bcbc f   wavedev2_common_topaz_v1:hwctxt.obj
 0001:0000acd8       ?CallHPDetectInterruptThread@@YAXPAVHardwareContext@@@Z 1000bcd8 f   wavedev2_common_topaz_v1:hwctxt.obj
 0001:0000acf4       ?SetOutputGain@HardwareContext@@QAAIK@Z 1000bcf4 f   wavedev2_common_topaz_v1:hwctxt.obj
 0001:0000ad34       ?SetOutputMute@HardwareContext@@QAAIH@Z 1000bd34 f   wavedev2_common_topaz_v1:hwctxt.obj
 0001:0000ad74       ?GetOutputGain@HardwareContext@@QAAKXZ 1000bd74 f   wavedev2_common_topaz_v1:hwctxt.obj
 0001:0000ada4       ?GetOutputMute@HardwareContext@@QAAHXZ 1000bda4 f   wavedev2_common_topaz_v1:hwctxt.obj
 0001:0000add4       ?GetInputMute@HardwareContext@@QAAHXZ 1000bdd4 f   wavedev2_common_topaz_v1:hwctxt.obj
 0001:0000ae04       ?SetInputMute@HardwareContext@@QAAIH@Z 1000be04 f   wavedev2_common_topaz_v1:hwctxt.obj
 0001:0000ae44       ?GetInputGain@HardwareContext@@QAAKXZ 1000be44 f   wavedev2_common_topaz_v1:hwctxt.obj
 0001:0000ae74       ?SetInputGain@HardwareContext@@QAAIK@Z 1000be74 f   wavedev2_common_topaz_v1:hwctxt.obj
 0001:0000aeb4       ?SetSpeakerEnable@HardwareContext@@IAAXH@Z 1000beb4 f   wavedev2_common_topaz_v1:hwctxt.obj
 0001:0000aed0       ?RecalcSpeakerEnable@HardwareContext@@IAAXXZ 1000bed0 f   wavedev2_common_topaz_v1:hwctxt.obj
 0001:0000aef8       ?ForceSpeaker@HardwareContext@@QAAKH@Z 1000bef8 f   wavedev2_common_topaz_v1:hwctxt.obj
 0001:0000afa0       ?PmControlMessage@HardwareContext@@QAAHKPAEK0KPAK@Z 1000bfa0 f   wavedev2_common_topaz_v1:hwctxt.obj
 0001:0000b3b4       ?PowerUp@HardwareContext@@QAAXXZ 1000c3b4 f   wavedev2_common_topaz_v1:hwctxt.obj
 0001:0000b430       ?PowerDown@HardwareContext@@QAAXXZ 1000c430 f   wavedev2_common_topaz_v1:hwctxt.obj
 0001:0000b524       ?GetDriverRegValue@HardwareContext@@QAAKPAGK@Z 1000c524 f   wavedev2_common_topaz_v1:hwctxt.obj
 0001:0000b5a4       ?SetDriverRegValue@HardwareContext@@QAAXPAGK@Z 1000c5a4 f   wavedev2_common_topaz_v1:hwctxt.obj
 0001:0000b610       ?IsSupportedOutputFormat@HardwareContext@@QAAHPAUtWAVEFORMATEX@@@Z 1000c610 f   wavedev2_common_topaz_v1:hwctxt.obj
 0001:0000b640       ?SelectInputSource@HardwareContext@@QAAHK@Z 1000c640 f   wavedev2_common_topaz_v1:hwctxt.obj
 0001:0000b6c0       ?SetCodecLoopback@HardwareContext@@QAAHH@Z 1000c6c0 f   wavedev2_common_topaz_v1:hwctxt.obj
 0001:0000b7e0       ??0InputDeviceContext@@QAA@XZ 1000c7e0 f i wavedev2_common_topaz_v1:hwctxt.obj
 0001:0000b820       ??0OutputDeviceContext@@QAA@XZ 1000c820 f i wavedev2_common_topaz_v1:hwctxt.obj
 0001:0000b860       SetEvent                   1000c860 f i wavedev2_common_topaz_v1:hwctxt.obj
 0001:0000b898       ?GetInterruptThreadPriority@HardwareContext@@IAAKXZ 1000c898 f i wavedev2_common_topaz_v1:hwctxt.obj
 0001:0000b8d8       ?UpdateOutputGain@HardwareContext@@IAAXXZ 1000c8d8 f i wavedev2_common_topaz_v1:hwctxt.obj
 0001:0000b92c       ?UpdateInputGain@HardwareContext@@IAAXXZ 1000c92c f i wavedev2_common_topaz_v1:hwctxt.obj
 0001:0000b980       ??0DeviceContext@@QAA@XZ   1000c980 f   wavedev2_common_topaz_v1:devctxt.obj
 0001:0000ba6c       ?GetGain@DeviceContext@@QAAKXZ 1000ca6c f   wavedev2_common_topaz_v1:devctxt.obj
 0001:0000ba9c       ?SetGain@DeviceContext@@QAAKK@Z 1000ca9c f   wavedev2_common_topaz_v1:devctxt.obj
 0001:0000badc       ?GetDefaultStreamGain@DeviceContext@@QAAKXZ 1000cadc f   wavedev2_common_topaz_v1:devctxt.obj
 0001:0000bb0c       ?SetDefaultStreamGain@DeviceContext@@QAAKK@Z 1000cb0c f   wavedev2_common_topaz_v1:devctxt.obj
 0001:0000bb44       ?GetSecondaryGainLimit@DeviceContext@@QAAKK@Z 1000cb44 f   wavedev2_common_topaz_v1:devctxt.obj
 0001:0000bb84       ?SetSecondaryGainLimit@DeviceContext@@QAAKKK@Z 1000cb84 f   wavedev2_common_topaz_v1:devctxt.obj
 0001:0000bbec       ?IsSupportedFormat@DeviceContext@@UAAHPAUtWAVEFORMATEX@@@Z 1000cbec f   wavedev2_common_topaz_v1:devctxt.obj
 0001:0000be88       ?IsSupportedFormat@OutputDeviceContext@@UAAHPAUtWAVEFORMATEX@@@Z 1000ce88 f   wavedev2_common_topaz_v1:devctxt.obj
 0001:0000bf20       ?NewStream@DeviceContext@@UAAKPAVStreamContext@@@Z 1000cf20 f   wavedev2_common_topaz_v1:devctxt.obj
 0001:0000c064       ?DeleteStream@DeviceContext@@QAAXPAVStreamContext@@@Z 1000d064 f   wavedev2_common_topaz_v1:devctxt.obj
 0001:0000c0fc       ?TransferBuffer@DeviceContext@@QAAPAEPAE0PAUTRANSFER_STATUS@@@Z 1000d0fc f   wavedev2_common_topaz_v1:devctxt.obj
 0001:0000c20c       ?RecalcAllGains@DeviceContext@@QAAXXZ 1000d20c f   wavedev2_common_topaz_v1:devctxt.obj
 0001:0000c288       ?StreamReadyToRender@OutputDeviceContext@@UAAXPAVStreamContext@@@Z 1000d288 f   wavedev2_common_topaz_v1:devctxt.obj
 0001:0000c2ac       ?StreamReadyToRender@InputDeviceContext@@UAAXPAVStreamContext@@@Z 1000d2ac f   wavedev2_common_topaz_v1:devctxt.obj
 0001:0000c2d0       ?GetDevCaps@OutputDeviceContext@@UAAKPAXK@Z 1000d2d0 f   wavedev2_common_topaz_v1:devctxt.obj
 0001:0000c348       ?GetDevCaps@InputDeviceContext@@UAAKPAXK@Z 1000d348 f   wavedev2_common_topaz_v1:devctxt.obj
 0001:0000c3c0       ?GetExtDevCaps@OutputDeviceContext@@UAAKPAXK@Z 1000d3c0 f   wavedev2_common_topaz_v1:devctxt.obj
 0001:0000c410       ?GetExtDevCaps@InputDeviceContext@@UAAKPAXK@Z 1000d410 f   wavedev2_common_topaz_v1:devctxt.obj
 0001:0000c438       ?CreateStream@InputDeviceContext@@UAAPAVStreamContext@@PAUwaveopendesc_tag@@@Z 1000d438 f   wavedev2_common_topaz_v1:devctxt.obj
 0001:0000c4a0       ?CreateStream@OutputDeviceContext@@UAAPAVStreamContext@@PAUwaveopendesc_tag@@@Z 1000d4a0 f   wavedev2_common_topaz_v1:devctxt.obj
 0001:0000cafc       ?OpenStream@DeviceContext@@QAAKPAUwaveopendesc_tag@@KPAPAVStreamContext@@@Z 1000dafc f   wavedev2_common_topaz_v1:devctxt.obj
 0001:0000cce4       ?SetBaseSampleRate@DeviceContext@@UAAXK@Z 1000dce4 f   wavedev2_common_topaz_v1:devctxt.obj
 0001:0000cd34       ?ResetBaseInfo@DeviceContext@@QAAXXZ 1000dd34 f   wavedev2_common_topaz_v1:devctxt.obj
 0001:0000cdb0       ?GetBaseSampleRate@DeviceContext@@QAAKXZ 1000ddb0 f   wavedev2_common_topaz_v1:devctxt.obj
 0001:0000cde0       ?GetBaseSampleRateInverse@DeviceContext@@QAAKXZ 1000dde0 f   wavedev2_common_topaz_v1:devctxt.obj
 0001:0000ce10       ?GetChannels@OutputDeviceContext@@UAAKXZ 1000de10 f   wavedev2_common_topaz_v1:devctxt.obj
 0001:0000ce38       ?GetChannels@InputDeviceContext@@UAAKXZ 1000de38 f   wavedev2_common_topaz_v1:devctxt.obj
 0001:0000ce60       ?GetNativeFormat@DeviceContext@@QAAKKPAXKPAK@Z 1000de60 f   wavedev2_common_topaz_v1:devctxt.obj
 0001:0000cf98       ?GetProperty@DeviceContext@@QAAKPAUtag_WAVEPROPINFO@@@Z 1000df98 f   wavedev2_common_topaz_v1:devctxt.obj
 0001:0000d0e8       ?SetProperty@DeviceContext@@QAAKPAUtag_WAVEPROPINFO@@@Z 1000e0e8 f   wavedev2_common_topaz_v1:devctxt.obj
 0001:0000d118       ??0InputStreamContext@@QAA@XZ 1000e118 f i wavedev2_common_topaz_v1:devctxt.obj
 0001:0000d15c       ??_GInputStreamContext@@UAAPAXI@Z 1000e15c f i wavedev2_common_topaz_v1:devctxt.obj
 0001:0000d15c       ??_EInputStreamContext@@UAAPAXI@Z 1000e15c f i wavedev2_common_topaz_v1:devctxt.obj
 0001:0000d1a0       ??0WaveStreamContext@@QAA@XZ 1000e1a0 f i wavedev2_common_topaz_v1:devctxt.obj
 0001:0000d1e4       ??1InputStreamContext@@UAA@XZ 1000e1e4 f i wavedev2_common_topaz_v1:devctxt.obj
 0001:0000d200       ??1WaveStreamContext@@UAA@XZ 1000e200 f i wavedev2_common_topaz_v1:devctxt.obj
 0001:0000d21c       ??_EWaveStreamContext@@UAAPAXI@Z 1000e21c f i wavedev2_common_topaz_v1:devctxt.obj
 0001:0000d21c       ??_GWaveStreamContext@@UAAPAXI@Z 1000e21c f i wavedev2_common_topaz_v1:devctxt.obj
 0001:0000d260       ??0CMidiStream@@QAA@XZ     1000e260 f i wavedev2_common_topaz_v1:devctxt.obj
 0001:0000d2a4       ??0OutputStreamContext16bitM8@@QAA@XZ 1000e2a4 f i wavedev2_common_topaz_v1:devctxt.obj
 0001:0000d2e8       ??0OutputStreamContext16bitS8@@QAA@XZ 1000e2e8 f i wavedev2_common_topaz_v1:devctxt.obj
 0001:0000d32c       ??0OutputStreamContext16bitM16@@QAA@XZ 1000e32c f i wavedev2_common_topaz_v1:devctxt.obj
 0001:0000d370       ??0OutputStreamContext16bitS16@@QAA@XZ 1000e370 f i wavedev2_common_topaz_v1:devctxt.obj
 0001:0000d3b4       ??0OutputStreamContext24bitM8@@QAA@XZ 1000e3b4 f i wavedev2_common_topaz_v1:devctxt.obj
 0001:0000d3f8       ??0OutputStreamContext24bitS8@@QAA@XZ 1000e3f8 f i wavedev2_common_topaz_v1:devctxt.obj
 0001:0000d43c       ??0OutputStreamContext24bitM16@@QAA@XZ 1000e43c f i wavedev2_common_topaz_v1:devctxt.obj
 0001:0000d480       ??0OutputStreamContext24bitS16@@QAA@XZ 1000e480 f i wavedev2_common_topaz_v1:devctxt.obj
 0001:0000d4c4       ??0OutputStreamContext24bitS24@@QAA@XZ 1000e4c4 f i wavedev2_common_topaz_v1:devctxt.obj
 0001:0000d508       ??_GCMidiStream@@UAAPAXI@Z 1000e508 f i wavedev2_common_topaz_v1:devctxt.obj
 0001:0000d508       ??_ECMidiStream@@UAAPAXI@Z 1000e508 f i wavedev2_common_topaz_v1:devctxt.obj
 0001:0000d54c       ??_GOutputStreamContext16bitM8@@UAAPAXI@Z 1000e54c f i wavedev2_common_topaz_v1:devctxt.obj
 0001:0000d54c       ??_EOutputStreamContext16bitM8@@UAAPAXI@Z 1000e54c f i wavedev2_common_topaz_v1:devctxt.obj
 0001:0000d590       ??0OutputStreamContext@@QAA@XZ 1000e590 f i wavedev2_common_topaz_v1:devctxt.obj
 0001:0000d5d4       ??_EOutputStreamContext16bitS8@@UAAPAXI@Z 1000e5d4 f i wavedev2_common_topaz_v1:devctxt.obj
 0001:0000d5d4       ??_GOutputStreamContext16bitS8@@UAAPAXI@Z 1000e5d4 f i wavedev2_common_topaz_v1:devctxt.obj
 0001:0000d618       ??_GOutputStreamContext16bitM16@@UAAPAXI@Z 1000e618 f i wavedev2_common_topaz_v1:devctxt.obj
 0001:0000d618       ??_EOutputStreamContext16bitM16@@UAAPAXI@Z 1000e618 f i wavedev2_common_topaz_v1:devctxt.obj
 0001:0000d65c       ??_EOutputStreamContext16bitS16@@UAAPAXI@Z 1000e65c f i wavedev2_common_topaz_v1:devctxt.obj
 0001:0000d65c       ??_GOutputStreamContext16bitS16@@UAAPAXI@Z 1000e65c f i wavedev2_common_topaz_v1:devctxt.obj
 0001:0000d6a0       ??_GOutputStreamContext24bitM8@@UAAPAXI@Z 1000e6a0 f i wavedev2_common_topaz_v1:devctxt.obj
 0001:0000d6a0       ??_EOutputStreamContext24bitM8@@UAAPAXI@Z 1000e6a0 f i wavedev2_common_topaz_v1:devctxt.obj
 0001:0000d6e4       ??_GOutputStreamContext24bitS8@@UAAPAXI@Z 1000e6e4 f i wavedev2_common_topaz_v1:devctxt.obj
 0001:0000d6e4       ??_EOutputStreamContext24bitS8@@UAAPAXI@Z 1000e6e4 f i wavedev2_common_topaz_v1:devctxt.obj
 0001:0000d728       ??_GOutputStreamContext24bitM16@@UAAPAXI@Z 1000e728 f i wavedev2_common_topaz_v1:devctxt.obj
 0001:0000d728       ??_EOutputStreamContext24bitM16@@UAAPAXI@Z 1000e728 f i wavedev2_common_topaz_v1:devctxt.obj
 0001:0000d76c       ??_GOutputStreamContext24bitS16@@UAAPAXI@Z 1000e76c f i wavedev2_common_topaz_v1:devctxt.obj
 0001:0000d76c       ??_EOutputStreamContext24bitS16@@UAAPAXI@Z 1000e76c f i wavedev2_common_topaz_v1:devctxt.obj
 0001:0000d7b0       ??_GOutputStreamContext24bitS24@@UAAPAXI@Z 1000e7b0 f i wavedev2_common_topaz_v1:devctxt.obj
 0001:0000d7b0       ??_EOutputStreamContext24bitS24@@UAAPAXI@Z 1000e7b0 f i wavedev2_common_topaz_v1:devctxt.obj
 0001:0000d7f4       ??1CMidiStream@@UAA@XZ     1000e7f4 f i wavedev2_common_topaz_v1:devctxt.obj
 0001:0000d810       ??1OutputStreamContext16bitM8@@UAA@XZ 1000e810 f i wavedev2_common_topaz_v1:devctxt.obj
 0001:0000d82c       ??1OutputStreamContext@@UAA@XZ 1000e82c f i wavedev2_common_topaz_v1:devctxt.obj
 0001:0000d848       ??_GOutputStreamContext@@UAAPAXI@Z 1000e848 f i wavedev2_common_topaz_v1:devctxt.obj
 0001:0000d848       ??_EOutputStreamContext@@UAAPAXI@Z 1000e848 f i wavedev2_common_topaz_v1:devctxt.obj
 0001:0000d88c       ??1OutputStreamContext16bitS8@@UAA@XZ 1000e88c f i wavedev2_common_topaz_v1:devctxt.obj
 0001:0000d8a8       ??1OutputStreamContext16bitM16@@UAA@XZ 1000e8a8 f i wavedev2_common_topaz_v1:devctxt.obj
 0001:0000d8c4       ??1OutputStreamContext16bitS16@@UAA@XZ 1000e8c4 f i wavedev2_common_topaz_v1:devctxt.obj
 0001:0000d8e0       ??1OutputStreamContext24bitM8@@UAA@XZ 1000e8e0 f i wavedev2_common_topaz_v1:devctxt.obj
 0001:0000d8fc       ??1OutputStreamContext24bitS8@@UAA@XZ 1000e8fc f i wavedev2_common_topaz_v1:devctxt.obj
 0001:0000d918       ??1OutputStreamContext24bitM16@@UAA@XZ 1000e918 f i wavedev2_common_topaz_v1:devctxt.obj
 0001:0000d934       ??1OutputStreamContext24bitS16@@UAA@XZ 1000e934 f i wavedev2_common_topaz_v1:devctxt.obj
 0001:0000d950       ??1OutputStreamContext24bitS24@@UAA@XZ 1000e950 f i wavedev2_common_topaz_v1:devctxt.obj
 0001:0000d96c       ?IsEqualGUID@@YAHABU_GUID@@0@Z 1000e96c f i wavedev2_common_topaz_v1:devctxt.obj
 0001:0000d9c8       ??0StreamContext@@QAA@XZ   1000e9c8 f   wavedev2_common_topaz_v1:strmctxt.obj
 0001:0000da00       ??1StreamContext@@UAA@XZ   1000ea00 f   wavedev2_common_topaz_v1:strmctxt.obj
 0001:0000da24       ?StillPlaying@StreamContext@@QAAHXZ 1000ea24 f   wavedev2_common_topaz_v1:strmctxt.obj
 0001:0000da74       ?GetByteCount@StreamContext@@QAAKXZ 1000ea74 f   wavedev2_common_topaz_v1:strmctxt.obj
 0001:0000daa4       ?GetWaveFormat@StreamContext@@QAAPAUtWAVEFORMATEX@@XZ 1000eaa4 f   wavedev2_common_topaz_v1:strmctxt.obj
 0001:0000dad0       ?GetDeviceContext@StreamContext@@QAAPAVDeviceContext@@XZ 1000ead0 f   wavedev2_common_topaz_v1:strmctxt.obj
 0001:0000db00       ?DoDriverCallback@StreamContext@@QAAXIKK@Z 1000eb00 f   wavedev2_common_topaz_v1:strmctxt.obj
 0001:0000db58       ?DoCallbackReturnBuffer@StreamContext@@UAAXPAUwavehdr_tag@@@Z 1000eb58 f   wavedev2_common_topaz_v1:strmctxt.obj
 0001:0000db84       ?DoCallbackStreamOpened@StreamContext@@UAAXXZ 1000eb84 f   wavedev2_common_topaz_v1:strmctxt.obj
 0001:0000dbb0       ?DoCallbackStreamClosed@StreamContext@@UAAXXZ 1000ebb0 f   wavedev2_common_topaz_v1:strmctxt.obj
 0001:0000dbd8       ?ReturnBuffer@StreamContext@@QAAXPAUwavehdr_tag@@@Z 1000ebd8 f   wavedev2_common_topaz_v1:strmctxt.obj
 0001:0000dc48       ?GetGain@StreamContext@@QAAKXZ 1000ec48 f   wavedev2_common_topaz_v1:strmctxt.obj
 0001:0000dc78       ?SetGain@StreamContext@@QAAKK@Z 1000ec78 f   wavedev2_common_topaz_v1:strmctxt.obj
 0001:0000dccc       ?SetSecondaryGainClass@StreamContext@@QAAKK@Z 1000eccc f   wavedev2_common_topaz_v1:strmctxt.obj
 0001:0000dd38       ?GainChange@StreamContext@@UAAXXZ 1000ed38 f   wavedev2_common_topaz_v1:strmctxt.obj
 0001:0000ddb8       ?IsExclusive@StreamContext@@UAAHXZ 1000edb8 f   wavedev2_common_topaz_v1:strmctxt.obj
 0001:0000dde0       ?Open@StreamContext@@UAAKPAVDeviceContext@@PAUwaveopendesc_tag@@K@Z 1000ede0 f   wavedev2_common_topaz_v1:strmctxt.obj
 0001:0000e0b8       ?Close@StreamContext@@UAAKXZ 1000f0b8 f   wavedev2_common_topaz_v1:strmctxt.obj
 0001:0000e12c       ?AddRef@StreamContext@@QAAJXZ 1000f12c f   wavedev2_common_topaz_v1:strmctxt.obj
 0001:0000e180       ?Release@StreamContext@@QAAJXZ 1000f180 f   wavedev2_common_topaz_v1:strmctxt.obj
 0001:0000e244       ?QueueBuffer@StreamContext@@UAAKPAUwavehdr_tag@@@Z 1000f244 f   wavedev2_common_topaz_v1:strmctxt.obj
 0001:0000e404       ?GetNextBuffer@StreamContext@@QAAPAEXZ 1000f404 f   wavedev2_common_topaz_v1:strmctxt.obj
 0001:0000e5e4       ?BreakLoop@StreamContext@@QAAKXZ 1000f5e4 f   wavedev2_common_topaz_v1:strmctxt.obj
 0001:0000e6c0       ?MapGain@StreamContext@@QAAKKK@Z 1000f6c0 f   wavedev2_common_topaz_v1:strmctxt.obj
 0001:0000e8d4       ?GetPos@StreamContext@@UAAKPAUmmtime_tag@@@Z 1000f8d4 f   wavedev2_common_topaz_v1:strmctxt.obj
 0001:0000eb08       ?Open@WaveStreamContext@@UAAKPAVDeviceContext@@PAUwaveopendesc_tag@@K@Z 1000fb08 f   wavedev2_common_topaz_v1:strmctxt.obj
 0001:0000edd0       ?GetRate@WaveStreamContext@@QAAKPAK@Z 1000fdd0 f   wavedev2_common_topaz_v1:strmctxt.obj
 0001:0000ee0c       ?Run@StreamContext@@UAAKXZ 1000fe0c f   wavedev2_common_topaz_v1:strmctxt.obj
 0001:0000ee88       ?Stop@StreamContext@@UAAKXZ 1000fe88 f   wavedev2_common_topaz_v1:strmctxt.obj
 0001:0000eec0       ?Reset@StreamContext@@UAAKXZ 1000fec0 f   wavedev2_common_topaz_v1:strmctxt.obj
 0001:0000efd4       ?ForceSpeaker@StreamContext@@QAAKH@Z 1000ffd4 f   wavedev2_common_topaz_v1:strmctxt.obj
 0001:0000f070       ?SetRate@WaveStreamContext@@UAAKK@Z 10010070 f   wavedev2_common_topaz_v1:strmctxt.obj
 0001:0000f190       ?Render@WaveStreamContext@@UAAPAEPAE00PAUTRANSFER_STATUS@@@Z 10010190 f   wavedev2_common_topaz_v1:strmctxt.obj
 0001:0000f2ec       ?ClearBuffer@StreamContext@@SAXPAE0@Z 100102ec f   wavedev2_common_topaz_v1:strmctxt.obj
 0001:0000f318       ?GetProperty@StreamContext@@QAAKPAUtag_WAVEPROPINFO@@@Z 10010318 f   wavedev2_common_topaz_v1:strmctxt.obj
 0001:0000f358       ?SetProperty@StreamContext@@QAAKPAUtag_WAVEPROPINFO@@@Z 10010358 f   wavedev2_common_topaz_v1:strmctxt.obj
 0001:0000f398       ??_EStreamContext@@UAAPAXI@Z 10010398 f i wavedev2_common_topaz_v1:strmctxt.obj
 0001:0000f398       ??_GStreamContext@@UAAPAXI@Z 10010398 f i wavedev2_common_topaz_v1:strmctxt.obj
 0001:0000f3dc       ?COMPTYPE@@YAPAGK@Z        100103dc f   wavedev2_common_topaz_v1:mixerdrv.obj
 0001:0000f47c       ?LookupMxLine@@YAPBUtagMXLINEDESC@@G@Z 1001047c f   wavedev2_common_topaz_v1:mixerdrv.obj
 0001:0000f518       ?PerformMixerCallbacks@@YAXKK@Z 10010518 f   wavedev2_common_topaz_v1:mixerdrv.obj
 0001:0000f5e4       ?wdev_MXDM_GETDEVCAPS@@YAKPAUtagMIXERCAPS@@K@Z 100105e4 f   wavedev2_common_topaz_v1:mixerdrv.obj
 0001:0000f6dc       ?wdev_MXDM_OPEN@@YAKPAKPAUtMIXEROPENDESC@@K@Z 100106dc f   wavedev2_common_topaz_v1:mixerdrv.obj
 0001:0000f828       ?wdev_MXDM_CLOSE@@YAKK@Z   10010828 f   wavedev2_common_topaz_v1:mixerdrv.obj
 0001:0000f8ec       ?wdev_MXDM_GETLINEINFO@@YAKPAUtMIXERLINE@@K@Z 100108ec f   wavedev2_common_topaz_v1:mixerdrv.obj
 0001:000104d0       ?wdev_MXDM_GETLINECONTROLS@@YAKPAUtMIXERLINECONTROLS@@K@Z 100114d0 f   wavedev2_common_topaz_v1:mixerdrv.obj
 0001:00010bcc       ?wdev_MXDM_GETCONTROLDETAILS@@YAKPAUtMIXERCONTROLDETAILS@@K@Z 10011bcc f   wavedev2_common_topaz_v1:mixerdrv.obj
 0001:00010ce8       ?wdev_MXDM_SETCONTROLDETAILS@@YAKPAUtMIXERCONTROLDETAILS@@K@Z 10011ce8 f   wavedev2_common_topaz_v1:mixerdrv.obj
 0001:00010e3c       ?InitMixerControls@@YAHXZ  10011e3c f   wavedev2_common_topaz_v1:mixerdrv.obj
 0001:00010eb4       ?HandleMixerMessage@@YAHPAUMMDRV_MESSAGE_PARAMS@@PAK@Z 10011eb4 f   wavedev2_common_topaz_v1:mixerdrv.obj
 0001:00011260       ?SetMasterVolume@@YAIK@Z   10012260 f   wavedev2_common_topaz_v1:mixerdrv.obj
 0001:000112e0       ?GetMasterVolume@@YAKXZ    100122e0 f   wavedev2_common_topaz_v1:mixerdrv.obj
 0001:00011334       ?LookupControlByIndex@MixerControlList@@QAAPAVMixerControl@@K@Z 10012334 f i wavedev2_common_topaz_v1:mixerdrv.obj
 0001:0001138c       ??0MixerControlList@@QAA@XZ 1001238c f i wavedev2_common_topaz_v1:mixerdrv.obj
 0001:00011514       ??0MixerControlVolumeMaster@@QAA@XZ 10012514 f i wavedev2_common_topaz_v1:mixerdrv.obj
 0001:00011558       ?SetControlID@MixerControl@@UAAXK@Z 10012558 f i wavedev2_common_topaz_v1:mixerdrv.obj
 0001:0001157c       ??0MixerControlVolume@@QAA@XZ 1001257c f i wavedev2_common_topaz_v1:mixerdrv.obj
 0001:000115c0       ??0MixerControl@@QAA@XZ    100125c0 f i wavedev2_common_topaz_v1:mixerdrv.obj
 0001:00011608       ?CopyMixerControl@MixerControl@@UAAXPAUtMIXERCONTROL@@@Z 10012608 f i wavedev2_common_topaz_v1:mixerdrv.obj
 0001:000116dc       ?GetControlID@MixerControl@@QAAKXZ 100126dc f i wavedev2_common_topaz_v1:mixerdrv.obj
 0001:0001170c       ?GetControlDetails@MixerControl@@UAAKPAUtMIXERCONTROLDETAILS@@K@Z 1001270c f i wavedev2_common_topaz_v1:mixerdrv.obj
 0001:00011734       ?SetControlDetails@MixerControl@@UAAKPAUtMIXERCONTROLDETAILS@@K@Z 10012734 f i wavedev2_common_topaz_v1:mixerdrv.obj
 0001:0001175c       ??_GMixerControl@@UAAPAXI@Z 1001275c f i wavedev2_common_topaz_v1:mixerdrv.obj
 0001:0001175c       ??_EMixerControl@@UAAPAXI@Z 1001275c f i wavedev2_common_topaz_v1:mixerdrv.obj
 0001:000117a0       ??1MixerControl@@UAA@XZ    100127a0 f i wavedev2_common_topaz_v1:mixerdrv.obj
 0001:000117c4       ?CopyMixerControl@MixerControlVolume@@UAAXPAUtMIXERCONTROL@@@Z 100127c4 f i wavedev2_common_topaz_v1:mixerdrv.obj
 0001:000118d8       ?GetControlType@MixerControlVolume@@UAAKXZ 100128d8 f i wavedev2_common_topaz_v1:mixerdrv.obj
 0001:00011904       ?GetControlDetails@MixerControlVolume@@UAAKPAUtMIXERCONTROLDETAILS@@K@Z 10012904 f i wavedev2_common_topaz_v1:mixerdrv.obj
 0001:00011adc       ?SetControlDetails@MixerControlVolume@@UAAKPAUtMIXERCONTROLDETAILS@@K@Z 10012adc f i wavedev2_common_topaz_v1:mixerdrv.obj
 0001:00011ce8       ??_GMixerControlVolume@@UAAPAXI@Z 10012ce8 f i wavedev2_common_topaz_v1:mixerdrv.obj
 0001:00011ce8       ??_EMixerControlVolume@@UAAPAXI@Z 10012ce8 f i wavedev2_common_topaz_v1:mixerdrv.obj
 0001:00011d2c       ??1MixerControlVolume@@UAA@XZ 10012d2c f i wavedev2_common_topaz_v1:mixerdrv.obj
 0001:00011d48       ?CopyMixerControl@MixerControlVolumeMaster@@UAAXPAUtMIXERCONTROL@@@Z 10012d48 f i wavedev2_common_topaz_v1:mixerdrv.obj
 0001:00011d8c       ?GetLineID@MixerControlVolumeMaster@@UAAGXZ 10012d8c f i wavedev2_common_topaz_v1:mixerdrv.obj
 0001:00011db8       ?SetGain@MixerControlVolumeMaster@@UAAXK@Z 10012db8 f i wavedev2_common_topaz_v1:mixerdrv.obj
 0001:00011de0       ?GetGain@MixerControlVolumeMaster@@UAAKXZ 10012de0 f i wavedev2_common_topaz_v1:mixerdrv.obj
 0001:00011e1c       ??_GMixerControlVolumeMaster@@UAAPAXI@Z 10012e1c f i wavedev2_common_topaz_v1:mixerdrv.obj
 0001:00011e1c       ??_EMixerControlVolumeMaster@@UAAPAXI@Z 10012e1c f i wavedev2_common_topaz_v1:mixerdrv.obj
 0001:00011e60       ??1MixerControlVolumeMaster@@UAA@XZ 10012e60 f i wavedev2_common_topaz_v1:mixerdrv.obj
 0001:00011e7c       ??0MixerControlVolumeMic@@QAA@XZ 10012e7c f i wavedev2_common_topaz_v1:mixerdrv.obj
 0001:00011ec0       ?CopyMixerControl@MixerControlVolumeMic@@UAAXPAUtMIXERCONTROL@@@Z 10012ec0 f i wavedev2_common_topaz_v1:mixerdrv.obj
 0001:00011f04       ?GetLineID@MixerControlVolumeMic@@UAAGXZ 10012f04 f i wavedev2_common_topaz_v1:mixerdrv.obj
 0001:00011f30       ?SetGain@MixerControlVolumeMic@@UAAXK@Z 10012f30 f i wavedev2_common_topaz_v1:mixerdrv.obj
 0001:00011f58       ?GetGain@MixerControlVolumeMic@@UAAKXZ 10012f58 f i wavedev2_common_topaz_v1:mixerdrv.obj
 0001:00011f94       ??_GMixerControlVolumeMic@@UAAPAXI@Z 10012f94 f i wavedev2_common_topaz_v1:mixerdrv.obj
 0001:00011f94       ??_EMixerControlVolumeMic@@UAAPAXI@Z 10012f94 f i wavedev2_common_topaz_v1:mixerdrv.obj
 0001:00011fd8       ??1MixerControlVolumeMic@@UAA@XZ 10012fd8 f i wavedev2_common_topaz_v1:mixerdrv.obj
 0001:00011ff4       ??0MixerControlMuteMaster@@QAA@XZ 10012ff4 f i wavedev2_common_topaz_v1:mixerdrv.obj
 0001:00012038       ??0MixerControlBoolean@@QAA@XZ 10013038 f i wavedev2_common_topaz_v1:mixerdrv.obj
 0001:0001207c       ?CopyMixerControl@MixerControlBoolean@@UAAXPAUtMIXERCONTROL@@@Z 1001307c f i wavedev2_common_topaz_v1:mixerdrv.obj
 0001:0001218c       ?GetControlType@MixerControlBoolean@@UAAKXZ 1001318c f i wavedev2_common_topaz_v1:mixerdrv.obj
 0001:000121b8       ?GetControlDetails@MixerControlBoolean@@UAAKPAUtMIXERCONTROLDETAILS@@K@Z 100131b8 f i wavedev2_common_topaz_v1:mixerdrv.obj
 0001:00012268       ?SetControlDetails@MixerControlBoolean@@UAAKPAUtMIXERCONTROLDETAILS@@K@Z 10013268 f i wavedev2_common_topaz_v1:mixerdrv.obj
 0001:0001230c       ??_EMixerControlBoolean@@UAAPAXI@Z 1001330c f i wavedev2_common_topaz_v1:mixerdrv.obj
 0001:0001230c       ??_GMixerControlBoolean@@UAAPAXI@Z 1001330c f i wavedev2_common_topaz_v1:mixerdrv.obj
 0001:00012350       ??1MixerControlBoolean@@UAA@XZ 10013350 f i wavedev2_common_topaz_v1:mixerdrv.obj
 0001:0001236c       ?CopyMixerControl@MixerControlMuteMaster@@UAAXPAUtMIXERCONTROL@@@Z 1001336c f i wavedev2_common_topaz_v1:mixerdrv.obj
 0001:000123b0       ?GetControlType@MixerControlMuteMaster@@UAAKXZ 100133b0 f i wavedev2_common_topaz_v1:mixerdrv.obj
 0001:000123dc       ?GetLineID@MixerControlMuteMaster@@UAAGXZ 100133dc f i wavedev2_common_topaz_v1:mixerdrv.obj
 0001:00012408       ?GetValue@MixerControlMuteMaster@@UAAHXZ 10013408 f i wavedev2_common_topaz_v1:mixerdrv.obj
 0001:00012444       ?SetValue@MixerControlMuteMaster@@UAAXH@Z 10013444 f i wavedev2_common_topaz_v1:mixerdrv.obj
 0001:0001246c       ??_GMixerControlMuteMaster@@UAAPAXI@Z 1001346c f i wavedev2_common_topaz_v1:mixerdrv.obj
 0001:0001246c       ??_EMixerControlMuteMaster@@UAAPAXI@Z 1001346c f i wavedev2_common_topaz_v1:mixerdrv.obj
 0001:000124b0       ??1MixerControlMuteMaster@@UAA@XZ 100134b0 f i wavedev2_common_topaz_v1:mixerdrv.obj
 0001:000124cc       ??0MixerControlMuteMic@@QAA@XZ 100134cc f i wavedev2_common_topaz_v1:mixerdrv.obj
 0001:00012510       ?CopyMixerControl@MixerControlMuteMic@@UAAXPAUtMIXERCONTROL@@@Z 10013510 f i wavedev2_common_topaz_v1:mixerdrv.obj
 0001:00012554       ?GetLineID@MixerControlMuteMic@@UAAGXZ 10013554 f i wavedev2_common_topaz_v1:mixerdrv.obj
 0001:00012580       ?GetValue@MixerControlMuteMic@@UAAHXZ 10013580 f i wavedev2_common_topaz_v1:mixerdrv.obj
 0001:000125bc       ?SetValue@MixerControlMuteMic@@UAAXH@Z 100135bc f i wavedev2_common_topaz_v1:mixerdrv.obj
 0001:000125e4       ??_GMixerControlMuteMic@@UAAPAXI@Z 100135e4 f i wavedev2_common_topaz_v1:mixerdrv.obj
 0001:000125e4       ??_EMixerControlMuteMic@@UAAPAXI@Z 100135e4 f i wavedev2_common_topaz_v1:mixerdrv.obj
 0001:00012628       ??1MixerControlMuteMic@@UAA@XZ 10013628 f i wavedev2_common_topaz_v1:mixerdrv.obj
 0001:00012644       ??0MixerControlLoopback@@QAA@XZ 10013644 f i wavedev2_common_topaz_v1:mixerdrv.obj
 0001:00012698       ?CopyMixerControl@MixerControlLoopback@@UAAXPAUtMIXERCONTROL@@@Z 10013698 f i wavedev2_common_topaz_v1:mixerdrv.obj
 0001:000126e0       ?GetControlType@MixerControlLoopback@@UAAKXZ 100136e0 f i wavedev2_common_topaz_v1:mixerdrv.obj
 0001:0001270c       ?GetLineID@MixerControlLoopback@@UAAGXZ 1001370c f i wavedev2_common_topaz_v1:mixerdrv.obj
 0001:00012738       ?GetValue@MixerControlLoopback@@UAAHXZ 10013738 f i wavedev2_common_topaz_v1:mixerdrv.obj
 0001:00012768       ?SetValue@MixerControlLoopback@@UAAXH@Z 10013768 f i wavedev2_common_topaz_v1:mixerdrv.obj
 0001:000127d4       ??_GMixerControlLoopback@@UAAPAXI@Z 100137d4 f i wavedev2_common_topaz_v1:mixerdrv.obj
 0001:000127d4       ??_EMixerControlLoopback@@UAAPAXI@Z 100137d4 f i wavedev2_common_topaz_v1:mixerdrv.obj
 0001:00012818       ??1MixerControlLoopback@@UAA@XZ 10013818 f i wavedev2_common_topaz_v1:mixerdrv.obj
 0001:00012834       ??0MixerControlInputMux@@QAA@XZ 10013834 f i wavedev2_common_topaz_v1:mixerdrv.obj
 0001:00012888       ?CopyMixerControl@MixerControlInputMux@@UAAXPAUtMIXERCONTROL@@@Z 10013888 f i wavedev2_common_topaz_v1:mixerdrv.obj
 0001:000129d0       ?GetLineID@MixerControlInputMux@@UAAGXZ 100139d0 f i wavedev2_common_topaz_v1:mixerdrv.obj
 0001:000129fc       ?GetControlType@MixerControlInputMux@@UAAKXZ 100139fc f i wavedev2_common_topaz_v1:mixerdrv.obj
 0001:00012a28       ?GetNumSelections@MixerControlInputMux@@QAAKXZ 10013a28 f i wavedev2_common_topaz_v1:mixerdrv.obj
 0001:00012a50       ?GetControlDetails@MixerControlInputMux@@UAAKPAUtMIXERCONTROLDETAILS@@K@Z 10013a50 f i wavedev2_common_topaz_v1:mixerdrv.obj
 0001:00012ca0       ?GetListText@MixerControlInputMux@@QAAXPAUtMIXERCONTROLDETAILS_LISTTEXT@@K@Z 10013ca0 f i wavedev2_common_topaz_v1:mixerdrv.obj
 0001:00012da8       ?GetComponentType@MixerControl@@QAAKXZ 10013da8 f i wavedev2_common_topaz_v1:mixerdrv.obj
 0001:00012e10       ?GetCurrSelection@MixerControlInputMux@@QAAKK@Z 10013e10 f i wavedev2_common_topaz_v1:mixerdrv.obj
 0001:00012e64       ?SetControlDetails@MixerControlInputMux@@UAAKPAUtMIXERCONTROLDETAILS@@K@Z 10013e64 f i wavedev2_common_topaz_v1:mixerdrv.obj
 0001:00012fe4       ?SetCurrSelection@MixerControlInputMux@@QAAXKH@Z 10013fe4 f i wavedev2_common_topaz_v1:mixerdrv.obj
 0001:0001305c       ??_GMixerControlInputMux@@UAAPAXI@Z 1001405c f i wavedev2_common_topaz_v1:mixerdrv.obj
 0001:0001305c       ??_EMixerControlInputMux@@UAAPAXI@Z 1001405c f i wavedev2_common_topaz_v1:mixerdrv.obj
 0001:000130a0       ??1MixerControlInputMux@@UAA@XZ 100140a0 f i wavedev2_common_topaz_v1:mixerdrv.obj
 0001:000130bc       ??_EMixerControlList@@UAAPAXI@Z 100140bc f i wavedev2_common_topaz_v1:mixerdrv.obj
 0001:000130bc       ??_GMixerControlList@@UAAPAXI@Z 100140bc f i wavedev2_common_topaz_v1:mixerdrv.obj
 0001:00013100       ??1MixerControlList@@UAA@XZ 10014100 f i wavedev2_common_topaz_v1:mixerdrv.obj
 0001:0001316c       ?Open@InputStreamContext@@UAAKPAVDeviceContext@@PAUwaveopendesc_tag@@K@Z 1001416c f   wavedev2_common_topaz_v1:input.obj
 0001:000131d0       ?DoCallbackReturnBuffer@InputStreamContext@@UAAXPAUwavehdr_tag@@@Z 100141d0 f   wavedev2_common_topaz_v1:input.obj
 0001:000131f8       ?DoCallbackStreamOpened@InputStreamContext@@UAAXXZ 100141f8 f   wavedev2_common_topaz_v1:input.obj
 0001:00013224       ?DoCallbackStreamClosed@InputStreamContext@@UAAXXZ 10014224 f   wavedev2_common_topaz_v1:input.obj
 0001:00013250       ?Stop@InputStreamContext@@UAAKXZ 10014250 f   wavedev2_common_topaz_v1:input.obj
 0001:000132b8       ?Render2@InputStreamContext@@UAAPAEPAE00PAUTRANSFER_STATUS@@@Z 100142b8 f   wavedev2_common_topaz_v1:input.obj
 0001:0001398c       ?ResetBaseInfo@InputStreamContext@@UAAXXZ 1001498c f   wavedev2_common_topaz_v1:input.obj
 0001:000139a0       ?GainChange@CMidiStream@@UAAXXZ 100149a0 f   wavedev2_common_topaz_v1:midistrm.obj
 0001:00013a08       ?MapNoteGain@CMidiStream@@QAAKKK@Z 10014a08 f   wavedev2_common_topaz_v1:midistrm.obj
 0001:00013ad8       ?Open@CMidiStream@@UAAKPAVDeviceContext@@PAUwaveopendesc_tag@@K@Z 10014ad8 f   wavedev2_common_topaz_v1:midistrm.obj
 0001:00013d4c       ?Reset@CMidiStream@@UAAKXZ 10014d4c f   wavedev2_common_topaz_v1:midistrm.obj
 0001:00013dbc       ?Close@CMidiStream@@UAAKXZ 10014dbc f   wavedev2_common_topaz_v1:midistrm.obj
 0001:00013e10       ?UpdateTempo@CMidiStream@@QAAJXZ 10014e10 f   wavedev2_common_topaz_v1:midistrm.obj
 0001:00013f84       ?ProcessMidiStream@CMidiStream@@QAAIXZ 10014f84 f   wavedev2_common_topaz_v1:midistrm.obj
 0001:00014104       ?Render@CMidiStream@@UAAPAEPAE00PAUTRANSFER_STATUS@@@Z 10015104 f   wavedev2_common_topaz_v1:midistrm.obj
 0001:0001435c       ?MidiMessage@CMidiStream@@QAAKI@Z 1001535c f   wavedev2_common_topaz_v1:midistrm.obj
 0001:00014424       ?InternalMidiMessage@CMidiStream@@QAAJI@Z 10015424 f   wavedev2_common_topaz_v1:midistrm.obj
 0001:00014580       ?MidiData@CMidiStream@@QAAJI@Z 10015580 f   wavedev2_common_topaz_v1:midistrm.obj
 0001:000146d8       ?FindNote@CMidiStream@@QAAPAVCMidiNote@@II@Z 100156d8 f   wavedev2_common_topaz_v1:midistrm.obj
 0001:00014788       ?NoteOn@CMidiStream@@QAAJIII@Z 10015788 f   wavedev2_common_topaz_v1:midistrm.obj
 0001:00014874       ?NoteOff@CMidiStream@@QAAJIII@Z 10015874 f   wavedev2_common_topaz_v1:midistrm.obj
 0001:000148d0       ?AllNotesOff@CMidiStream@@QAAJI@Z 100158d0 f   wavedev2_common_topaz_v1:midistrm.obj
 0001:00014948       ?ResetBaseInfo@CMidiStream@@UAAXXZ 10015948 f   wavedev2_common_topaz_v1:midistrm.obj
 0001:00014ac8       ?GetDeltaFromNote@CMidiStream@@QAAKK@Z 10015ac8 f   wavedev2_common_topaz_v1:midistrm.obj
 0001:00014b6c       ?GetDeltaFromFreq@CMidiStream@@QAAKK@Z 10015b6c f   wavedev2_common_topaz_v1:midistrm.obj
 0001:00014bb8       ?NoteMoveToFreeList@CMidiStream@@QAAXPAVCMidiNote@@@Z 10015bb8 f   wavedev2_common_topaz_v1:midistrm.obj
 0001:00014c70       ?NoteMoveToNoteList@CMidiStream@@QAAXPAVCMidiNote@@@Z 10015c70 f   wavedev2_common_topaz_v1:midistrm.obj
 0001:00014d28       ?NoteDone@CMidiStream@@QAAXPAVCMidiNote@@@Z 10015d28 f   wavedev2_common_topaz_v1:midistrm.obj
 0001:00014d50       ?DeltaTicksToSamples@CMidiStream@@QAAII@Z 10015d50 f   wavedev2_common_topaz_v1:midistrm.obj
 0001:00014d8c       ?Open@OutputStreamContext@@UAAKPAVDeviceContext@@PAUwaveopendesc_tag@@K@Z 10015d8c f   wavedev2_common_topaz_v1:output.obj
 0001:00014e24       ?Reset@OutputStreamContext@@UAAKXZ 10015e24 f   wavedev2_common_topaz_v1:output.obj
 0001:00014e88       ?ResetBaseInfo@OutputStreamContext@@UAAXXZ 10015e88 f   wavedev2_common_topaz_v1:output.obj
 0001:00014e9c       ?Render2@OutputStreamContext16bitM8@@UAAPAEPAE00PAUTRANSFER_STATUS@@@Z 10015e9c f   wavedev2_common_topaz_v1:output.obj
 0001:0001520c       ?Render2@OutputStreamContext16bitM16@@UAAPAEPAE00PAUTRANSFER_STATUS@@@Z 1001620c f   wavedev2_common_topaz_v1:output.obj
 0001:0001556c       ?Render2@OutputStreamContext16bitS8@@UAAPAEPAE00PAUTRANSFER_STATUS@@@Z 1001656c f   wavedev2_common_topaz_v1:output.obj
 0001:00015970       ?Render2@OutputStreamContext16bitS16@@UAAPAEPAE00PAUTRANSFER_STATUS@@@Z 10016970 f   wavedev2_common_topaz_v1:output.obj
 0001:00015ed8       ?Render2@OutputStreamContextMC@@UAAPAEPAE00PAUTRANSFER_STATUS@@@Z 10016ed8 f   wavedev2_common_topaz_v1:output.obj
 0001:00016554       ?Render2@OutputStreamContext24bitM8@@UAAPAEPAE00PAUTRANSFER_STATUS@@@Z 10017554 f   wavedev2_common_topaz_v1:output.obj
 0001:00016a2c       ?Render2@OutputStreamContext24bitM16@@UAAPAEPAE00PAUTRANSFER_STATUS@@@Z 10017a2c f   wavedev2_common_topaz_v1:output.obj
 0001:00016ea4       ?Render2@OutputStreamContext24bitS8@@UAAPAEPAE00PAUTRANSFER_STATUS@@@Z 10017ea4 f   wavedev2_common_topaz_v1:output.obj
 0001:00017414       ?Render2@OutputStreamContext24bitS16@@UAAPAEPAE00PAUTRANSFER_STATUS@@@Z 10018414 f   wavedev2_common_topaz_v1:output.obj
 0001:00017c30       ?Render2@OutputStreamContext24bitS24@@UAAPAEPAE00PAUTRANSFER_STATUS@@@Z 10018c30 f   wavedev2_common_topaz_v1:output.obj
 0001:00018200       ?GainChange@CMidiNote@@QAAXXZ 10019200 f   wavedev2_common_topaz_v1:midinote.obj
 0001:00018288       ?ResetBaseInfo@CMidiNote@@QAAXXZ 10019288 f   wavedev2_common_topaz_v1:midinote.obj
 0001:0001831c       ?NoteOn@CMidiNote@@QAAJPAVCMidiStream@@III@Z 1001931c f   wavedev2_common_topaz_v1:midinote.obj
 0001:00018398       ?NoteOff@CMidiNote@@QAAJI@Z 10019398 f   wavedev2_common_topaz_v1:midinote.obj
 0001:000184ac       ?Render@CMidiNote@@QAAPAEPAE00PAUTRANSFER_STATUS@@@Z 100194ac f   wavedev2_common_topaz_v1:midinote.obj
 0001:00018610       ?Render2@CMidiNote@@QAAPAEPAE00PAUTRANSFER_STATUS@@@Z 10019610 f   wavedev2_common_topaz_v1:midinote.obj
 0001:00018a58       ?NoteVal@CMidiNote@@QAAIXZ 10019a58 f   wavedev2_common_topaz_v1:midinote.obj
 0001:00018a88       ?NoteChannel@CMidiNote@@QAAIXZ 10019a88 f   wavedev2_common_topaz_v1:midinote.obj
 0001:00018ab8       ?SetVelocity@CMidiNote@@QAAXI@Z 10019ab8 f   wavedev2_common_topaz_v1:midinote.obj
 0001:00018b08       ?GetSsiBaseRegAddr@@YAII@Z 10019b08 f   wavedev2_mx25_topaz_v1:csphwctxt.obj
 0001:00018b74       ?GetAudmuxBaseRegAddr@@YAIXZ 10019b74 f   wavedev2_mx25_topaz_v1:csphwctxt.obj
 0001:00018b90       ?GetSdmaChannelIRQ@@YAKI@Z 10019b90 f   wavedev2_mx25_topaz_v1:csphwctxt.obj
 0001:00018bbc       NKDbgPrintfW               10019bbc f   coredll:COREDLL.dll
 0001:00018bcc       InitializeCriticalSection  10019bcc f   coredll:COREDLL.dll
 0001:00018bdc       DeleteCriticalSection      10019bdc f   coredll:COREDLL.dll
 0001:00018bec       LeaveCriticalSection       10019bec f   coredll:COREDLL.dll
 0001:00018bfc       EnterCriticalSection       10019bfc f   coredll:COREDLL.dll
 0001:00018c0c       Sleep                      10019c0c f   coredll:COREDLL.dll
 0001:00018c1c       DisableThreadLibraryCalls  10019c1c f   coredll:COREDLL.dll
 0001:00018c2c       RegisterDbgZones           10019c2c f   coredll:COREDLL.dll
 0001:00018c3c       SetLastError               10019c3c f   coredll:COREDLL.dll
 0001:00018c4c       CeGetCallerTrust           10019c4c f   coredll:COREDLL.dll
 0001:00018c5c       CloseHandle                10019c5c f   coredll:COREDLL.dll
 0001:00018c6c       KernelIoControl            10019c6c f   coredll:COREDLL.dll
 0001:00018c7c       EventModify                10019c7c f   coredll:COREDLL.dll
 0001:00018c8c       CeSetThreadPriority        10019c8c f   coredll:COREDLL.dll
 0001:00018c9c       CreateThread               10019c9c f   coredll:COREDLL.dll
 0001:00018cac       InterruptInitialize        10019cac f   coredll:COREDLL.dll
 0001:00018cbc       CreateEventW               10019cbc f   coredll:COREDLL.dll
 0001:00018ccc       WaitForSingleObject        10019ccc f   coredll:COREDLL.dll
 0001:00018cdc       InterruptDone              10019cdc f   coredll:COREDLL.dll
 0001:00018cec       WaitForMultipleObjects     10019cec f   coredll:COREDLL.dll
 0001:00018cfc       RegCloseKey                10019cfc f   coredll:COREDLL.dll
 0001:00018d0c       RegQueryValueExW           10019d0c f   coredll:COREDLL.dll
 0001:00018d1c       OpenDeviceKey              10019d1c f   coredll:COREDLL.dll
 0001:00018d2c       RegSetValueExW             10019d2c f   coredll:COREDLL.dll
 0001:00018d3c       CeSafeCopyMemory           10019d3c f   coredll:COREDLL.dll
 0001:00018d4c       LocalAlloc                 10019d4c f   coredll:COREDLL.dll
 0001:00018d5c       LocalFree                  10019d5c f   coredll:COREDLL.dll
 0001:00018d6c       MmMapIoSpace               10019d6c f   ceddk:CEDDK.dll
 0001:00018d7c       HalAllocateCommonBuffer    10019d7c f   ceddk:CEDDK.dll
 0001:00018d8c       HalFreeCommonBuffer        10019d8c f   ceddk:CEDDK.dll
 0001:00018d9c       MmUnmapIoSpace             10019d9c f   ceddk:CEDDK.dll
 0001:00018dac       timeSetEvent               10019dac f   mmtimer:MMTimer.dll
 0001:00018dbc       timeKillEvent              10019dbc f   mmtimer:MMTimer.dll
 0001:00018dcc       DDKIomuxSetPinMux          10019dcc f   cspddk:CSPDDK.dll
 0001:00018ddc       DDKClockSetGatingMode      10019ddc f   cspddk:CSPDDK.dll
 0001:00018dec       DDKClockSetCKO             10019dec f   cspddk:CSPDDK.dll
 0001:00018dfc       DDKSdmaSetBufDesc          10019dfc f   cspddk:CSPDDK.dll
 0001:00018e0c       DDKSdmaAllocChain          10019e0c f   cspddk:CSPDDK.dll
 0001:00018e1c       DDKSdmaOpenChan            10019e1c f   cspddk:CSPDDK.dll
 0001:00018e2c       DDKSdmaStartChan           10019e2c f   cspddk:CSPDDK.dll
 0001:00018e3c       DDKSdmaInitChain           10019e3c f   cspddk:CSPDDK.dll
 0001:00018e4c       DDKSdmaStopChan            10019e4c f   cspddk:CSPDDK.dll
 0001:00018e5c       DDKSdmaClearBufDescStatus  10019e5c f   cspddk:CSPDDK.dll
 0001:00018e6c       DDKSdmaGetChainStatus      10019e6c f   cspddk:CSPDDK.dll
 0001:00018e7c       I2CSetFrequency            10019e7c f   i2csdk:I2CSDK.dll
 0001:00018e8c       I2CSetMasterMode           10019e8c f   i2csdk:I2CSDK.dll
 0001:00018e9c       I2COpenHandle              10019e9c f   i2csdk:I2CSDK.dll
 0001:00018eac       I2CCloseHandle             10019eac f   i2csdk:I2CSDK.dll
 0001:00018ebc       I2CTransfer                10019ebc f   i2csdk:I2CSDK.dll
 0001:00018ecc       _DllMainCRTStartup         10019ecc f   corelib0:pegdmain.obj
 0001:00019074       __security_init_cookie     1001a074 f   corelib0:seccinit.obj
 0001:0001913c       exit                       1001a13c f   corelib0:cexit.obj
 0001:000192bc       _exit                      1001a2bc f   corelib0:cexit.obj
 0001:000192e0       _cexit                     1001a2e0 f   corelib0:cexit.obj
 0001:000192fc       _c_exit                    1001a2fc f   corelib0:cexit.obj
 0001:00019318       GetCurrentProcess          1001a318 f i corelib0:cexit.obj
 0001:00019330       _initterm                  1001a330 f   corelib0:crt0dat.obj
 0001:00019384       _cinit                     1001a384 f   corelib0:crt0dat.obj
 0001:000193c0       _onexit                    1001a3c0 f   corelib0:onexit.obj
 0001:000196c4       atexit                     1001a6c4 f   corelib0:onexit.obj
 0001:00019718       log                        1001a718 f   corelib1:COREDLL.dll
 0001:00019728       __utod                     1001a728 f   corelib1:COREDLL.dll
 0001:00019738       __subd                     1001a738 f   corelib1:COREDLL.dll
 0001:00019748       __muld                     1001a748 f   corelib1:COREDLL.dll
 0001:00019758       __divd                     1001a758 f   corelib1:COREDLL.dll
 0001:00019768       __addd                     1001a768 f   corelib1:COREDLL.dll
 0001:00019778       __dtou                     1001a778 f   corelib1:COREDLL.dll
 0001:00019788       memset                     1001a788 f   corelib1:COREDLL.dll
 0001:00019798       ??3@YAXPAX@Z               1001a798 f   corelib1:COREDLL.dll
 0001:000197a8       ??2@YAPAXI@Z               1001a7a8 f   corelib1:COREDLL.dll
 0001:000197b8       __rt_udiv                  1001a7b8 f   corelib1:COREDLL.dll
 0001:000197c8       __utos                     1001a7c8 f   corelib1:COREDLL.dll
 0001:000197d8       __divs                     1001a7d8 f   corelib1:COREDLL.dll
 0001:000197e8       __itos                     1001a7e8 f   corelib1:COREDLL.dll
 0001:000197f8       __subs                     1001a7f8 f   corelib1:COREDLL.dll
 0001:00019808       __muls                     1001a808 f   corelib1:COREDLL.dll
 0001:00019818       __stou                     1001a818 f   corelib1:COREDLL.dll
 0001:00019828       __C_specific_handler       1001a828 f   corelib1:COREDLL.dll
 0001:00019838       __rt_sdiv                  1001a838 f   corelib1:COREDLL.dll
 0001:00019848       _purecall                  1001a848 f   corelib1:COREDLL.dll
 0001:00019858       memcpy                     1001a858 f   corelib1:COREDLL.dll
 0001:00019868       __rt_sdiv64by64            1001a868 f   corelib1:COREDLL.dll
 0001:00019878       memcmp                     1001a878 f   corelib1:COREDLL.dll
 0001:00019888       wcscpy                     1001a888 f   corelib1:COREDLL.dll
 0001:00019898       __rt_udiv64by64            1001a898 f   corelib1:COREDLL.dll
 0001:000198a8       _XcptFilter                1001a8a8 f   corelib1:COREDLL.dll
 0001:000198b8       __security_gen_cookie2     1001a8b8 f   corelib1:COREDLL.dll
 0001:000198c8       free                       1001a8c8 f   corelib1:COREDLL.dll
 0001:000198d8       malloc                     1001a8d8 f   corelib1:COREDLL.dll
 0001:000198e8       realloc                    1001a8e8 f   corelib1:COREDLL.dll
 0001:000198f8       _msize                     1001a8f8 f   corelib1:COREDLL.dll
 0001:00019908       InterlockedExchange        1001a908 f   coredll:COREDLL.dll
 0001:00019918       TerminateProcess           1001a918 f   coredll:COREDLL.dll
 0001:00019928       InterlockedCompareExchange 1001a928 f   coredll:COREDLL.dll
 0001:000199b0       __IMPORT_DESCRIPTOR_COREDLL 1001a9b0     coredll:COREDLL.dll
 0001:000199c4       __IMPORT_DESCRIPTOR_CEDDK  1001a9c4     ceddk:CEDDK.dll
 0001:000199d8       __IMPORT_DESCRIPTOR_MMTimer 1001a9d8     mmtimer:MMTimer.dll
 0001:000199ec       __IMPORT_DESCRIPTOR_CSPDDK 1001a9ec     cspddk:CSPDDK.dll
 0001:00019a00       __IMPORT_DESCRIPTOR_I2CSDK 1001aa00     i2csdk:I2CSDK.dll
 0001:00019a14       __NULL_IMPORT_DESCRIPTOR   1001aa14     coredll:COREDLL.dll
 0002:00000000       __imp_HalFreeCommonBuffer  1001b000     ceddk:CEDDK.dll
 0002:00000004       __imp_HalAllocateCommonBuffer 1001b004     ceddk:CEDDK.dll
 0002:00000008       __imp_MmMapIoSpace         1001b008     ceddk:CEDDK.dll
 0002:0000000c       __imp_MmUnmapIoSpace       1001b00c     ceddk:CEDDK.dll
 0002:00000010       \177CEDDK_NULL_THUNK_DATA  1001b010     ceddk:CEDDK.dll
 0002:00000014       __imp_Sleep                1001b014     coredll:COREDLL.dll
 0002:00000018       __imp_DisableThreadLibraryCalls 1001b018     coredll:COREDLL.dll
 0002:0000001c       __imp_RegisterDbgZones     1001b01c     coredll:COREDLL.dll
 0002:00000020       __imp_SetLastError         1001b020     coredll:COREDLL.dll
 0002:00000024       __imp_CeGetCallerTrust     1001b024     coredll:COREDLL.dll
 0002:00000028       __imp_CloseHandle          1001b028     coredll:COREDLL.dll
 0002:0000002c       __imp_KernelIoControl      1001b02c     coredll:COREDLL.dll
 0002:00000030       __imp_EventModify          1001b030     coredll:COREDLL.dll
 0002:00000034       __imp_CeSetThreadPriority  1001b034     coredll:COREDLL.dll
 0002:00000038       __imp_CreateThread         1001b038     coredll:COREDLL.dll
 0002:0000003c       __imp_InterruptInitialize  1001b03c     coredll:COREDLL.dll
 0002:00000040       __imp_EnterCriticalSection 1001b040     coredll:COREDLL.dll
 0002:00000044       __imp_WaitForSingleObject  1001b044     coredll:COREDLL.dll
 0002:00000048       __imp_InterruptDone        1001b048     coredll:COREDLL.dll
 0002:0000004c       __imp_WaitForMultipleObjects 1001b04c     coredll:COREDLL.dll
 0002:00000050       __imp_RegCloseKey          1001b050     coredll:COREDLL.dll
 0002:00000054       __imp_RegQueryValueExW     1001b054     coredll:COREDLL.dll
 0002:00000058       __imp_OpenDeviceKey        1001b058     coredll:COREDLL.dll
 0002:0000005c       __imp_RegSetValueExW       1001b05c     coredll:COREDLL.dll
 0002:00000060       __imp_CeSafeCopyMemory     1001b060     coredll:COREDLL.dll
 0002:00000064       __imp_LocalAlloc           1001b064     coredll:COREDLL.dll
 0002:00000068       __imp_LocalFree            1001b068     coredll:COREDLL.dll
 0002:0000006c       __imp_LeaveCriticalSection 1001b06c     coredll:COREDLL.dll
 0002:00000070       __imp_DeleteCriticalSection 1001b070     coredll:COREDLL.dll
 0002:00000074       __imp_InitializeCriticalSection 1001b074     coredll:COREDLL.dll
 0002:00000078       __imp_CreateEventW         1001b078     coredll:COREDLL.dll
 0002:0000007c       __imp_NKDbgPrintfW         1001b07c     coredll:COREDLL.dll
 0002:00000080       __imp_TerminateProcess     1001b080     coredll:COREDLL.dll
 0002:00000084       __imp_InterlockedExchange  1001b084     coredll:COREDLL.dll
 0002:00000088       __imp__msize               1001b088     corelib1:COREDLL.dll
 0002:0000008c       __imp_realloc              1001b08c     corelib1:COREDLL.dll
 0002:00000090       __imp_malloc               1001b090     corelib1:COREDLL.dll
 0002:00000094       __imp_free                 1001b094     corelib1:COREDLL.dll
 0002:00000098       __imp___security_gen_cookie2 1001b098     corelib1:COREDLL.dll
 0002:0000009c       __imp__XcptFilter          1001b09c     corelib1:COREDLL.dll
 0002:000000a0       __imp___rt_udiv64by64      1001b0a0     corelib1:COREDLL.dll
 0002:000000a4       __imp_wcscpy               1001b0a4     corelib1:COREDLL.dll
 0002:000000a8       __imp_memcmp               1001b0a8     corelib1:COREDLL.dll
 0002:000000ac       __imp_InterlockedCompareExchange 1001b0ac     coredll:COREDLL.dll
 0002:000000b0       __imp___rt_sdiv64by64      1001b0b0     corelib1:COREDLL.dll
 0002:000000b4       __imp_memcpy               1001b0b4     corelib1:COREDLL.dll
 0002:000000b8       __imp__purecall            1001b0b8     corelib1:COREDLL.dll
 0002:000000bc       __imp___rt_sdiv            1001b0bc     corelib1:COREDLL.dll
 0002:000000c0       __imp___C_specific_handler 1001b0c0     corelib1:COREDLL.dll
 0002:000000c4       __imp___stou               1001b0c4     corelib1:COREDLL.dll
 0002:000000c8       __imp___muls               1001b0c8     corelib1:COREDLL.dll
 0002:000000cc       __imp___subs               1001b0cc     corelib1:COREDLL.dll
 0002:000000d0       __imp___itos               1001b0d0     corelib1:COREDLL.dll
 0002:000000d4       __imp_log                  1001b0d4     corelib1:COREDLL.dll
 0002:000000d8       __imp___utod               1001b0d8     corelib1:COREDLL.dll
 0002:000000dc       __imp___subd               1001b0dc     corelib1:COREDLL.dll
 0002:000000e0       __imp___muld               1001b0e0     corelib1:COREDLL.dll
 0002:000000e4       __imp___divd               1001b0e4     corelib1:COREDLL.dll
 0002:000000e8       __imp___addd               1001b0e8     corelib1:COREDLL.dll
 0002:000000ec       __imp___dtou               1001b0ec     corelib1:COREDLL.dll
 0002:000000f0       __imp_memset               1001b0f0     corelib1:COREDLL.dll
 0002:000000f4       __imp_??3@YAXPAX@Z         1001b0f4     corelib1:COREDLL.dll
 0002:000000f8       __imp_??2@YAPAXI@Z         1001b0f8     corelib1:COREDLL.dll
 0002:000000fc       __imp___rt_udiv            1001b0fc     corelib1:COREDLL.dll
 0002:00000100       __imp___utos               1001b100     corelib1:COREDLL.dll
 0002:00000104       __imp___divs               1001b104     corelib1:COREDLL.dll
 0002:00000108       \177COREDLL_NULL_THUNK_DATA 1001b108     coredll:COREDLL.dll
 0002:0000010c       __imp_DDKSdmaStartChan     1001b10c     cspddk:CSPDDK.dll
 0002:00000110       __imp_DDKIomuxSetPinMux    1001b110     cspddk:CSPDDK.dll
 0002:00000114       __imp_DDKClockSetGatingMode 1001b114     cspddk:CSPDDK.dll
 0002:00000118       __imp_DDKClockSetCKO       1001b118     cspddk:CSPDDK.dll
 0002:0000011c       __imp_DDKSdmaSetBufDesc    1001b11c     cspddk:CSPDDK.dll
 0002:00000120       __imp_DDKSdmaAllocChain    1001b120     cspddk:CSPDDK.dll
 0002:00000124       __imp_DDKSdmaGetChainStatus 1001b124     cspddk:CSPDDK.dll
 0002:00000128       __imp_DDKSdmaClearBufDescStatus 1001b128     cspddk:CSPDDK.dll
 0002:0000012c       __imp_DDKSdmaInitChain     1001b12c     cspddk:CSPDDK.dll
 0002:00000130       __imp_DDKSdmaStopChan      1001b130     cspddk:CSPDDK.dll
 0002:00000134       __imp_DDKSdmaOpenChan      1001b134     cspddk:CSPDDK.dll
 0002:00000138       \177CSPDDK_NULL_THUNK_DATA 1001b138     cspddk:CSPDDK.dll
 0002:0000013c       __imp_I2CSetFrequency      1001b13c     i2csdk:I2CSDK.dll
 0002:00000140       __imp_I2CSetMasterMode     1001b140     i2csdk:I2CSDK.dll
 0002:00000144       __imp_I2COpenHandle        1001b144     i2csdk:I2CSDK.dll
 0002:00000148       __imp_I2CCloseHandle       1001b148     i2csdk:I2CSDK.dll
 0002:0000014c       __imp_I2CTransfer          1001b14c     i2csdk:I2CSDK.dll
 0002:00000150       \177I2CSDK_NULL_THUNK_DATA 1001b150     i2csdk:I2CSDK.dll
 0002:00000154       __imp_timeSetEvent         1001b154     mmtimer:MMTimer.dll
 0002:00000158       __imp_timeKillEvent        1001b158     mmtimer:MMTimer.dll
 0002:0000015c       \177MMTimer_NULL_THUNK_DATA 1001b15c     mmtimer:MMTimer.dll
 0002:00000160       dpCurSettings              1001b160     wavedev2_common_topaz_v1:wavemain.obj
 0002:00000658       ?ctype_table@@3PAUMMSYSCODE@@A 1001b658     wavedev2_common_topaz_v1:mixerdrv.obj
 0002:00000748       ?szNames@?1??GetListText@MixerControlInputMux@@QAAXPAUtMIXERCONTROLDETAILS_LISTTEXT@@K@Z@4PAPBGA 1001b748     wavedev2_common_topaz_v1:mixerdrv.obj
 0002:00000750       __security_cookie          1001b750     corelib0:seccinit.obj
 0002:00000754       __security_cookie_complement 1001b754     corelib0:seccinit.obj
 0002:0000075c       ?g_BitsPerSample@@3GA      1001b75c     wavedev2_common_topaz_v1:hwctxt.obj
 0002:00000760       ?g_pHWContext@@3PAVHardwareContext@@A 1001b760     wavedev2_common_topaz_v1:hwctxt.obj
 0002:00000778       ?ms_PitchTable@CMidiStream@@0PAKA 1001b778     wavedev2_common_topaz_v1:midistrm.obj
 0002:000007a8       ?ms_PitchTableInverseSampleRate@CMidiStream@@0KA 1001b7a8     wavedev2_common_topaz_v1:midistrm.obj
 0002:000007ac       _exitflag                  1001b7ac     corelib0:cexit.obj
 0002:000007b0       __onexitend                1001b7b0     <common>
 0002:000007b4       __onexitbegin              1001b7b4     <common>
 0002:000007b8       g_pcsExit                  1001b7b8     <common>
 0002:000007bc       _pRawDllMain               1001b7bc     <common>

 entry point at        0001:00018ecc

 Static symbols

 0001:00018f20       _DllMainCRTStartupHelper   10019f20 f   corelib0:pegdmain.obj
 0001:00019160       doexit                     1001a160 f   corelib0:cexit.obj
 0001:0001941c       lockexit                   1001a41c f   corelib0:onexit.obj
 0001:000194b8       unlockexit                 1001a4b8 f   corelib0:onexit.obj
 0001:000194e4       _onexit_nolock             1001a4e4 f   corelib0:onexit.obj
